:020000040000FA
:06000000D4EF4BF01200EA
:06000800F5EF1DF01200EF
:06002A0006002298000010
:10003000B5020000460000001E9800002B040000DE
:10004000040000001A980000FB02000004000000F9
:10005000F8970000DB01000022000000F09700008C
:100060001D04000008000000EE970000FE000000E4
:04007000020000008A
:100110000D01006B040E005D55E20051260DF3CF7A
:1001200001FDF4CF02FD000E0127010E022301CDD7
:10013000E9FF02CDEAFFEF6A01CDE9FF02CDEAFF58
:10014000250EE926000EEA22EF9001CDE9FF02CD4F
:10015000EAFF250EE926000EEA22EF8201CDE9FF33
:1001600002CDEAFF250EE926000EEA22EF8401CD3A
:10017000E9FF02CDEAFF250EE926000EEA22EF98FC
:1001800001CDE9FF02CDEAFF250EE926000EEA22A5
:10019000EF9601CDE9FF02CDEAFF0F0EE926000E32
:1001A000EA22EF6801CDE9FF02CDEAFF210EE92640
:1001B000000EEA22700EEE6E170EEE6EEE6AEE6A1A
:1001C000002BA8D70101986B040E996F9A6B9B6B5B
:1001D0009C6B9D6B12000D01006B040E005D5EE2D6
:1001E0000051260DF3CF01FDF4CF02FD000E0127D3
:1001F000010E022301CDE9FF02CDEAFFEF50000915
:100200004BE101CDE9FF02CDEAFF010EEF6E01CD1A
:10021000E9FF02CDEAFF0B0E9EC1EBFF0C0E9FC162
:10022000EBFF01CDE9FF02CDEAFF0D0EEB6A0E0EEA
:10023000EB6A01CDE9FF02CDEAFFEE52060EE92698
:10024000000EEA22EE6AEE6AEE6AEE6A01CDE9FF7E
:1002500002CDEAFF250EE926000EEA22EF8001CD4D
:10026000E9FF02CDEAFF250EE926000EEA22EF960D
:1002700001CDE9FF02CDEAFF0F0EE926000EEA22CA
:10028000EF6801CDE9FF02CDEAFF250EE926000E59
:10029000EA22EF82005104D0002B9FD7FE0E00D03F
:1002A00012000D010A6B076B040E075D16E2075181
:1002B000260DF3CF08FDF4CF09FD000E0827010E2F
:1002C000092308CDE9FF09CDEAFFEF50000903E15A
:1002D000010E0A6F02D0072BE7D70A5102E1FE0E8A
:1002E000C5D00101982B000E992308CDE9FF09CD57
:1002F000EAFF0B0E98C1EBFF0C0E99C1EBFF880EC5
:10030000D8809855130E995503E2986B040E996F97
:1003100008CDE9FF09CDEAFF250EE926000EEA2205
:10032000EF9008CDE9FF09CDEAFF0D0EA2C1EBFF6A
:100330000E0EA3C1EBFF9A2B000E9B239C239D2343
:1003400008CDE9FF09CDEAFF140EE926000EEA22E6
:100350009AC1EEFF9BC1EEFF9CC1EEFF9DC1EEFF77
:1003600008CDE9FF09CDEAFF180EE926000EEA22C2
:10037000EE6AEE6AEE6AEE6A0A0EE66EE66AA0C100
:10038000E6FFA1C1E6FF08CDE9FF09CDEAFFEE5285
:10039000E9CF0BF0EACF0CF00BC0E6FF0CC0E6FF94
:1003A00083EC47F0F56E060EE15EF5500101C86B77
:1003B000C96B0101C7690101020EC66F08CDE9FFD3
:1003C00009CDEAFF180EE926000EEA22EECFC2F1AF
:1003D000EECFC3F1EECFC4F1EFCFC5F108CDE9FF09
:1003E00009CDEAFF140EE926000EEA22EECFBEF197
:1003F000EECFBFF1EECFC0F1EFCFC1F108CDE9FFF5
:1004000009CDEAFF0D0EE926000EEA22EECFBCF17F
:10041000EDCFBDF108CDE9FF09CDEAFF0B0EE926CE
:10042000000EEA22EECFBAF1EDCFBBF108CDE9FF25
:1004300009CDEAFFEE52E9CFB8F1EACFB9F196EC77
:1004400007F008CDE9FF09CDEAFF030EEF6E08CDF6
:10045000E9FF09CDEAFF140EE926000EEA22EE2A92
:10046000EE22EE22EE220D01075100D01200010112
:10047000A451260DF3CFE9FFF4CFEAFF000EE926E1
:10048000010EEA22EF50040802E0000E01D0010E36
:1004900000D012000101A551260DF3CF92FDF4CF3B
:1004A00093FD000E0D019227010E932392CDE9FFDB
:1004B00093CDEAFFEF50040807E092CDD2F193CD3F
:1004C000D3F1B6EC0AF061D0A5C1AAF1C9D90101F6
:1004D000C86BC96B0101C7690101110EC66F92CDCE
:1004E000E9FF93CDEAFF180EE926000EEA22EECFCF
:1004F000C2F1EECFC3F1EECFC4F1EFCFC5F192CD93
:10050000E9FF93CDEAFF140EE926000EEA22EECFB2
:10051000BEF1EECFBFF1EECFC0F1EFCFC1F192CD82
:10052000E9FF93CDEAFF0D0EE926000EEA22EECF99
:10053000BCF1EDCFBDF192CDE9FF93CDEAFF0B0EFB
:10054000E926000EEA22EECFBAF1EDCFBBF192CD53
:10055000E9FF93CDEAFFEE52E9CFB8F1EACFB9F166
:1005600096EC07F092CDE9FF93CDEAFF140EE92651
:10057000000EEA22EE2AEE22EE22EE2292CDE9FFD2
:1005800093CDEAFF050EEF6E00D012000101A651D7
:10059000260DF3CF96FDF4CF97FD000E0D019627A3
:1005A000010E972396CDE9FF97CDEAFF0F0EEB5092
:1005B000FF0802E1000EB5D096CDE9FF97CDEAFF26
:1005C000250EE926000EEA22EF50020B02E1000E92
:1005D000A8D096CDE9FF97CDEAFF100EE926000ED0
:1005E000EA22EECFC8F1EDCFC9F196CDE9FF97CD64
:1005F000EAFF0F0EEB500101C76F0101100EC66F2D
:1006000096CDE9FF97CDEAFF180EE926000EEA2203
:10061000EECFC2F1EECFC3F1EECFC4F1EFCFC5F113
:1006200096CDE9FF97CDEAFF140EE926000EEA22E7
:10063000EECFBEF1EECFBFF1EECFC0F1EFCFC1F103
:1006400096CDE9FF97CDEAFF0D0EE926000EEA22CE
:10065000EECFBCF1EDCFBDF196CDE9FF97CDEAFF2E
:100660000B0EE926000EEA22EECFBAF1EDCFBBF178
:1006700096CDE9FF97CDEAFFEE52E9CFB8F1EACF88
:10068000B9F196EC07F096CDE9FF97CDEAFF100E91
:10069000E926000EEA22EECF0BF0EFCF0CF00D6A48
:1006A0000E6A96CDE9FF97CDEAFF140EE926000EFB
:1006B000EA220B50EE260C50EE220D50EE220E5088
:1006C000EE2296CDE9FF97CDEAFF250EE926000E32
:1006D000EA22EF9296CDE9FF97CDEAFF250EE926B3
:1006E000000EEA22EF9896CDE9FF97CDEAFF0F0EB4
:1006F000EB500001E26F89EC2EF096CDE9FF97CD2B
:10070000EAFF0F0EE926000EEA22EF6896CDE9FF18
:1007100097CDEAFF250EE926000EEA22EF82010EB0
:1007200000D012000101A751260DF3CFE9FFF4CF4D
:10073000EAFF000EE926010EEA220F0EE926000E5E
:10074000EA22EF50FF0804E1B3EC2DF014D013D0EF
:10075000A751260DF3CFE9FFF4CFEAFF000EE926FB
:10076000010EEA22250EE926000EEA22EF50020BC6
:1007700001E0010E00D012000101A851260DF3CFB7
:1007800094FDF4CF95FD000E0D019427010E9523E5
:1007900094CDE9FF95CDEAFF0F0EEB50FF0826E15F
:1007A00094CDE9FF95CDEAFF0F0ED7C0EBFF94CDB6
:1007B000E9FF95CDEAFFEB500001E16F55EC2EF01B
:1007C00094CDE9FF95CDEAFF100EEB6A110EEB6AAE
:1007D000280E0001F26FF36B94CDE9FF95CDEAFF8F
:1007E0000F0EEB500001F16F37EC30F094CDE9FFC4
:1007F00095CDEAFF100EE926000EEA22EECF92FD1B
:10080000EDCF93FD0D01CA0E925D030E935902E3E5
:10081000000E25D094CDE9FF95CDEAFF250EE926FF
:10082000000EEA22EF88A9C1D8F0D6EC2DF00D0118
:10083000922B000E932394CDE9FF95CDEAFF100E85
:1008400092CDEBFF110E93CDEBFFCA0E925D030E1E
:10085000935903E3A8C1A6F199DE010E00D012005E
:100860000101AA51260DF3CF65FDF4CF66FD000E00
:100870000D016527010E662365CDE9FF66CDEAFF10
:10088000250EE926000EEA22EF50080B02E1000EC9
:100890000DD08CEC2EF065CDE9FF66CDEAFF250E7C
:1008A000E926000EEA22EF96010E00D012000101A7
:1008B000AB51260DF3CF00FDF4CF01FD000E0D016D
:1008C0000027010E012300CDE9FF01CDEAFF250E2F
:1008D000E926000EEA22EF50080B2FE000CDE9FFD9
:1008E00001CDEAFF250EE926000EEA22EF50040BA7
:1008F0000FE0280E0001EF6FF06B0CEC30F000CD34
:10090000E9FF01CDEAFF250EE926000EEA22EF9469
:1009100000CDE9FF01CDEAFF250EE926000EEA220F
:10092000EF88AEC1DFF0AFC1E0F0ACC1DDF0ADC12A
:10093000DEF02FEC2EF008D007D00B6A0C6A0BC04B
:10094000F3FF0CC0F4FF00D012000101B051260DDE
:10095000F3CF65FDF4CF66FD000E0D016527010E96
:10096000662365CDE9FF66CDEAFF250EE926000E78
:10097000EA22EF50080B44E065CDE9FF66CDEAFFBF
:10098000250EE926000EEA22EF50040B0FE0280E98
:100990000001EF6FF06B0CEC30F065CDE9FF66CD38
:1009A000EAFF250EE926000EEA22EF9465CDE9FF65
:1009B00066CDEAFF120EE926000EEA22EE50ED1097
:1009C0000CE18CEC2EF065CDE9FF66CDEAFF250E3B
:1009D000E926000EEA22EF9615D065CDE9FF66CD37
:1009E000EAFF120EE926000EEA22EE06EF5A10EC9C
:1009F0002EF0B1C1E9FFB2C1EAFFEF6E010E02D0E5
:100A0000000E00D012000101B351260DF3CFE9FF13
:100A1000F4CFEAFF000EE926010EEA22250EE926B0
:100A2000000EEA22EF50080B01E0010E00D0120088
:100A30000D010F6B006B040E005D01E36DD10051E1
:100A4000260DF3CF09FDF4CF0AFD000E0927010E94
:100A50000A2309CDE9FF0ACDEAFF250EE926000E9B
:100A6000EA22EF50080B0BE109CDE9FF0ACDEAFFBE
:100A7000250EE926000EEA22EF50100B01E049D1C5
:100A800009CDE9FF0ACDEAFFEF50000912E009CDD8
:100A9000E9FF0ACDEAFFEF5001080CE109CDE9FFBB
:100AA0000ACDEAFF250EE926000EEA22EF50010BDF
:100AB00001E02FD1A6EC4BF004C005FD05C006FDFA
:100AC00006C007FD07C008FD09CDE9FF0ACDEAFF12
:100AD0001D0EE926000EEA22EE500D01055D016FA4
:100AE000EE500659026FEE500759036FEE50085949
:100AF000046F09CDE9FF0ACDEAFF210EE926000EB9
:100B0000EA220151EE5C0251EE580351EE580451B5
:100B1000EE5801E3FED0B3EC2DF0000901E1FCD06A
:100B2000A6EC4BF004C00BF005C00CF006C00DF0B5
:100B300007C00EF009CDE9FF0ACDEAFF1D0EE92638
:100B4000000EEA220BC0EEFF0CC0EEFF0DC0EEFF60
:100B50000EC0EEFF09CDE9FF0ACDEAFF210EE9261E
:100B6000000EEA22EE2AEE22EE22EE2209CDE9FF65
:100B70000ACDEAFF1C0EE926000EEA22EF2A09CD73
:100B8000E9FF0ACDEAFFEF50060A43E0010A41E01F
:100B9000020A2CE00F0A2AE00E0A1EE0060A07E00D
:100BA000010A01E049D00D01020E0F6F45D009CDB9
:100BB000E9FF0ACDEAFF1C0EEB500B6E030E0B5C37
:100BC00004E20D01120E0F6F06D009CDD2F10ACD4D
:100BD000D3F1B6EC0AF030D00D01110E0F6F09CD34
:100BE000E9FF0ACDEAFF050EEF6E26D009CDE9FF39
:100BF0000ACDEAFF1C0EEB50030807E209CDD2F143
:100C00000ACDD3F1B6EC0AF003D00D01010E0F6F3F
:100C100013D009CDE9FF0ACDEAFF1C0EEB50030803
:100C200007E209CDD2F10ACDD3F1B6EC0AF003D038
:100C30000D01100E0F6F00D00D010F51000869E279
:100C4000100E0F5D15E009CDE9FF0ACDEAFF140E85
:100C5000E926000EEA22EFCF0BFDEE2AEFCF0CFDC6
:100C6000EE22EFCF0DFDEE22EFCF0EFDEF2210D0E2
:100C700009CDE9FF0ACDEAFF140EE926000EEA22AB
:100C8000EECF0BFDEECF0CFDEECF0DFDEFCF0EFD49
:100C90000101C86BC96B0101C7690FCDC6F109CD50
:100CA000E9FF0ACDEAFF180EE926000EEA22EECF90
:100CB000C2F1EECFC3F1EECFC4F1EFCFC5F10BCD52
:100CC000BEF10CCDBFF10DCDC0F10ECDC1F109CDFE
:100CD000E9FF0ACDEAFF0D0EE926000EEA22EECF6B
:100CE000BCF1EDCFBDF109CDE9FF0ACDEAFF0B0E56
:100CF000E926000EEA22EECFBAF1EDCFBBF109CD25
:100D0000E9FF0ACDEAFFEE52E9CFB8F1EACFB9F137
:100D10000DD90D01002B8FD61200140E0001DF6FCC
:100D2000E06B0001000EDD6F0D0EDE6F2FEC2EF07C
:100D30000101000ED06F0D0ED16F3DDBB4C1E9FF94
:100D4000B5C1EAFF060EE926000EEA22EECF14FD39
:100D5000EECF15FDEECF16FDEFCF17FD04C218FD47
:100D600005C219FD06C21AFD07C21BFD0D011C6B51
:100D7000060E1D6FB6C11EFDB7C11FFD1ECD0AF4C4
:100D80001FCD0BF46EEC48F0F3CF1EFDF4CF1FFD2A
:100D90000C0E0401126F136B0401140E106F0D0E74
:100DA000116FE6EC48F0F3CF21FDF4CF22FD0D01E9
:100DB000211F221F240E0001EF6FF06B0CEC30F0AE
:100DC00021CDD8F0D6EC2DF022CDD8F0D6EC2DF0F8
:100DD000140E0001EF6FF06B0CEC30F0B6C1CAF1ED
:100DE000B7C1CBF1A9D9F3CF21FDF4CF22FD0D017D
:100DF0001051211902E11151221904E08CEC2EF05E
:100E0000010E93D00C51F00BE842E842E842E84270
:100E1000040DF3500B6E0C6A140E0B5E000E0C5A90
:100E20000BC023FD23510B6E0C6A0B500101B65D04
:100E3000B66F0C50B759B76F140EB65F000EB75BA4
:100E40000D010C51F00BE842E842E842E842040D83
:100E5000F3500001EF6FF06B140EEF27000EF0233C
:100E60000CEC30F0B4C1CEF1B5C1CFF10101000EF0
:100E7000CC6F0D0ECD6F9BD90D01206FFE0E205D46
:100E800011E2B6C1D9F1B7C1DAF10101000ED76F95
:100E90000D0ED86FB4C1D5F1B5C1D6F120CDD4F1C6
:100EA000E4DB41D08CEC2EF0FF0E0D01205D3BE128
:100EB0000101B6510D0108270101B7510D010923A8
:100EC000000E0A230B230D51020B03E10D51010B00
:100ED00005E0082B000E09230A230B230101C86B30
:100EE000C96B0101C7690101040EC66F04CDC2F1CF
:100EF00005CDC3F106CDC4F107CDC5F108CDBEF1D6
:100F000009CDBFF10ACDC0F10BCDC1F100CDBCF1CF
:100F100001CDBDF102CDBAF103CDBBF1B4C1B8F141
:100F2000B5C1B9F103D8010E00D01200B3EC2DF019
:100F3000000901E1FBD7BAC167FDBBC168FDBCC1B7
:100F400069FDBDC16AFDBEC16BFDBFC16CFDC0C105
:100F50006DFDC1C16EFDC2C16FFDC3C170FDC4C1D5
:100F600071FDC5C172FD0D01749D749F73917393E2
:100F700073957397C6C174FDA0EC2EF0F3CF75FD89
:100F8000F4CF76FD0D01000E755D040E765904E375
:100F9000756B040E766F0DD0360ED8807555000E29
:100FA000765505E2360E755F000E765B02D0756BE6
:100FB000766B776B786B796B7A6B0101670ED06F0C
:100FC0000D0ED16FF8D9140E0101C827000EC923E8
:100FD000C6A310D0040EC827000EC9230D01020EAF
:100FE0007B6F040E7C6F7D6F7E6B7399738B738D3B
:100FF000739F05D00D017389739B738D739F04C21A
:101000007FFD05C280FD06C281FD07C282FDB8C119
:10101000E9FFB9C1EAFF060EE926000EEA22EECF8B
:1010200083FDEECF84FDEECF85FDEFCF86FD876B90
:10103000060E886FC8C189FDC9C18AFD89CD0AF431
:101040008ACD0BF46EEC48F0F3CF89FDF4CF8AFD26
:101050000C0E0401126F136B04017F0E106F0D0E46
:10106000116FE6EC48F0F3CF77FDF4CF78FD0D017A
:10107000771F781F77CD65FD78CD66FDFF0E0101E6
:10108000C75D02E1D7C0C7F1140E0001F26FF36B28
:10109000C7C1F1F037EC30F0C8C1FCF3C9C1FDF3B2
:1010A0000301060EFB6FB8C1F9F3B9C1FAF34AECBC
:1010B0003EF0140E0001DB6FDC6B0001670ED96F90
:1010C0000D0EDA6FF6EC2DF00101C6A30BD0040E65
:1010D0000001DB6FDC6B00017B0ED96F0D0EDA6F48
:1010E000F6EC2DF0140E0001F26FF36BC7C1F1F0B6
:1010F00037EC30F0C8C1CAF1C9C1CBF11DD8F3CF6C
:1011000065FDF4CF66FD240E0001F26FF36BC7C1DD
:10111000F1F037EC30F066CDD8F0D6EC2DF065CD9F
:10112000D8F0D6EC2DF00001F26BF36BC7C1F1F0F3
:1011300037EC30F0A5EF2FF00D01010E8B6F8C6BAB
:101140008D6B0101CAC10BF0CBC10CF0CA07000EB8
:10115000CB5B0B500C1020E010EC2EF00D018E6FCD
:101160008B510AE18E518C258C6F8E518C5D03E280
:101170008D2B01E18C2B09D08E518D258D6F8E51D9
:101180008D5D03E28C2B01E18D2B8B5102E0000E73
:1011900001D0010E8B6FD5D70D018D1D8D6F8C1D6C
:1011A0008C6F8CCDF3FF8DCDF4FF00D012000D01BC
:1011B000FE0E276F266B040E265D01E37FD02651BD
:1011C000260DF3CF24FDF4CF25FD000E2427010EBC
:1011D000252324CDE9FF25CDEAFFEF5000096BE080
:1011E00024CDE9FF25CDEAFF0B0EE926000EEA2209
:1011F000EECF0BF0EFCF0CF0CCC1E9FFCDC1EAFF91
:10120000020EE926000EEA22EECF0DF0EFCF0EF02F
:101210000D500B1802E10E500C184DE124CDE9FFE2
:1012200025CDEAFFEF50010802E126CD27FD24CDB0
:10123000E9FF25CDEAFF0D0EE926000EEA22EECFEA
:101240000BF0EFCF0CF0CCC1E9FFCDC1EAFFEECF40
:101250000DF0EFCF0EF00D500B1802E10E500C18F0
:101260002AE1CEC1E9FFCFC1EAFF060EE926000E52
:10127000EA22EECF0FF0EECF10F0EECF11F0EFCF6D
:1012800012F024CDE9FF25CDEAFFEE52060EE92645
:10129000000EEA22EE5000010F1909E1EE5010197C
:1012A00006E1EE50111903E1EE50121900E103E1DD
:1012B0000D0126517FD00D01262B7DD72751260DFC
:1012C000F3CF24FDF4CF25FD000E2427010E2523A6
:1012D000FE0E275D67E024CDE9FF25CDEAFFEF5044
:1012E000010860E10A0EE66EE66ACEC1E6FFCFC1F4
:1012F000E6FF24CDE9FF25CDEAFFEE52E9CF0BF062
:10130000EACF0CF00BC0E6FF0CC0E6FF83EC47F021
:10131000F56E060EE15EF550CCC1E9FFCDC1EAFFE6
:10132000020EE926000EEA22EECF0BF0EFCF0CF012
:1013300024CDE9FF25CDEAFF0B0E0BC0EBFF0C0E11
:101340000CC0EBFFCCC1E9FFCDC1EAFFEECF0BF043
:10135000EFCF0CF024CDE9FF25CDEAFF0D0E0BC039
:10136000EBFF0E0E0CC0EBFF24CDE9FF25CDEAFF0D
:10137000250EE926000EEA22EF9624CDE9FF25CDC1
:10138000EAFF0F0EE926000EEA22EF6824CDE9FFFE
:1013900025CDEAFF250EE926000EEA22EF820D0197
:1013A000275108D0FE0E275D03E1FF0E03D002D0C7
:1013B000FE0E00D01200D0C1E9FFD1C1EAFFEECF8E
:1013C0000AF4EDCF0BF46EEC48F0F3CF0BF0F4CF52
:1013D0000CF0D0C1E9FFD1C1EAFF0BC0EEFF0CC099
:1013E000EDFFD0C1E9FFD1C1EAFF020EE926000EF0
:1013F000EA22EECF0AF4EDCF0BF46EEC48F0F3CF17
:101400000BF0F4CF0CF0D0C1E9FFD1C1EAFF020E1E
:101410000BC0EBFF030E0CC0EBFFD0C1E9FFD1C145
:10142000EAFF040EE926000EEA22EECF0CF4EECF1E
:101430000DF4EECF0EF4EFCF0FF47EEC48F004C0C5
:101440000BF005C00CF006C00DF007C00EF0D0C1C7
:10145000E9FFD1C1EAFF040EE926000EEA220BC023
:10146000EEFF0CC0EEFF0DC0EEFF0EC0EEFFD0C1D0
:10147000E9FFD1C1EAFF080EE926000EEA22EECF0D
:101480000CF4EECF0DF4EECF0EF4EFCF0FF47EECB4
:1014900048F004C00BF005C00CF006C00DF007C00A
:1014A0000EF0D0C1E9FFD1C1EAFF080EE926000E17
:1014B000EA220BC0EEFF0CC0EEFF0DC0EEFF0EC027
:1014C000EEFFD0C1E9FFD1C1EAFF0E0EE926000E02
:1014D000EA22EECF0AF4EDCF0BF46EEC48F0F3CF36
:1014E0000BF0F4CF0CF0D0C1E9FFD1C1EAFF0E0E32
:1014F0000BC0EBFF0F0E0CC0EBFFD0C1E9FFD1C159
:10150000EAFF100EE926000EEA22EECF0AF4EDCF34
:101510000BF46EEC48F0F3CF0BF0F4CF0CF0D0C12D
:10152000E9FFD1C1EAFF100E0BC0EBFF110E0CC09A
:10153000EBFFD0C1E9FFD1C1EAFF120EE926000E90
:10154000EA22EECF0AF4EDCF0BF46EEC48F0F3CFC5
:101550000BF0F4CF0CF0D0C1E9FFD1C1EAFF120EBD
:101560000BC0EBFF130E0CC0EBFF1200D2C1E9FF62
:10157000D3C1EAFF0F0EEB50FF081CE0D2C1E9FF18
:10158000D3C1EAFF0F0EEB500001E26F89EC2EF0A1
:10159000D2C1E9FFD3C1EAFF0F0EE926000EEA220D
:1015A000EF68D2C1E9FFD3C1EAFF250EE926000E9C
:1015B000EA22EF82D2C1E9FFD3C1EAFFEE52060E62
:1015C000E926000EEA22EE6AEE6AEE6AEE6AD2C1FF
:1015D000E9FFD3C1EAFF0D0EEB6A0E0EEB6AD2C132
:1015E000E9FFD3C1EAFF250EE926000EEA22EF50FB
:1015F000080B02E08CEC2EF0D2C1E9FFD3C1EAFF68
:10160000250EE926000EEA22EF96D2C1E9FFD3C1EA
:10161000EAFF210EE926000EEA22700EEE6E170E8A
:10162000EE6EEE6AEE6AD2C1E9FFD3C1EAFF250E83
:10163000E926000EEA22EF98D2C1E9FFD3C1EAFF02
:10164000250EE926000EEA22EF50010B07E0D2C179
:10165000E9FFD3C1EAFF010EEF6E05D0D2C1E9FF69
:10166000D3C1EAFFEF6A00D012000D01366B010111
:10167000D451260DF3CF34FDF4CF35FD000E0D010E
:101680003427010E352334CDE9FF35CDEAFF180E9E
:10169000E926000EEA22EECF2CFDEECF2DFDEECF97
:1016A0002EFDEFCF2FFD34CDE9FF35CDEAFF140E2F
:1016B000E926000EEA22EECF30FDEECF31FDEECF6F
:1016C00032FDEFCF33FDD7C1E9FFD8C1EAFF040EE9
:1016D000E926000EEA22EECF24FDEECF25FDEECF67
:1016E00026FDEFCF27FD0101D9510D01242701016E
:1016F000DA510D012523000E2623272334CDE9FFDF
:1017000035CDEAFF140EE926000EEA22EECF28FDC1
:10171000EECF29FDEECF2AFDEFCF2BFD34CDE9FF33
:1017200035CDEAFF1C0EE926000EEA22EF6AA6EC90
:101730004BF004C00BF005C00CF006C00DF007C064
:101740000EF034CDE9FF35CDEAFF1D0EE926000E7F
:10175000EA220BC0EEFF0CC0EEFF0DC0EEFF0EC084
:10176000EEFF34CDE9FF35CDEAFF210EE926000E6C
:10177000EA22700EEE6E170EEE6EEE6AEE6A34CD51
:10178000E9FF35CDEAFFEF50010801E0B1D08CEC64
:101790002EF001019A2B000E9B239C239D2334CD18
:1017A000E9FF35CDEAFF140EE926000EEA229AC1C0
:1017B000EEFF9BC1EEFF9CC1EEFF9DC1EEFF0D0150
:1017C000242B25232623272334CDE9FF35CDEAFF1B
:1017D000180EE926000EEA2224CDEEFF25CDEEFFFD
:1017E00026CDEEFF27CDEEFF34CDE9FF35CDEAFF64
:1017F000140EE926000EEA22EECF28FDEECF29FDD9
:10180000EECF2AFDEFCF2BFD34CDE9FF35CDEAFF3A
:10181000140EE926000EEA22EE2AEE22EE22EE2235
:10182000D7C1E9FFD8C1EAFF0D0EE926000EEA2272
:10183000EF50020B36E00A0EE66EE66AD5C1E6FF0F
:10184000D6C1E6FF34CDE9FF35CDEAFFEE52E9CF50
:101850000BF0EACF0CF00BC0E6FF0CC0E6FF83EC08
:1018600047F0F56E060EE15EF550D7C1E9FFD8C12D
:10187000EAFFEECF0BF0EFCF0CF034CDE9FF35CD22
:10188000EAFF0D0E0BC0EBFF0E0E0CC0EBFF0D01BF
:10189000120E366F34CDE9FF35CDEAFF020EEF6E42
:1018A00026D0040E366F24CD28FD25CD29FD26CD6A
:1018B0002AFD27CD2BFDD7C1E9FFD8C1EAFFE926D4
:1018C000000EEA22EECF24FDEECF25FDEECF26FD61
:1018D000EFCF27FD34CDE9FF35CDEAFFEE52060EFE
:1018E000E926000EEA22EE6AEE6AEE6AEE6AA4D2F9
:1018F000D7C1E9FFD8C1EAFF0D0EE926000EEA22A2
:10190000EF50040B09E08CEC2EF034CDD2F135CD44
:10191000D3F12CDEC6D290D2D7C1E9FFD8C1EAFFFD
:10192000080EE926000EEA220D012851EE1809E101
:101930002951EE1806E12A51EE1803E12B51EE1859
:1019400000E101E077D234CDE9FF35CDEAFFEF5079
:1019500002086EE1D7C1E9FFD8C1EAFF0D0EE92602
:10196000000EEA22EF50100B60E034CDE9FF35CDD8
:10197000EAFF180EE926000EEA2224CDEEFF25CD5F
:10198000EEFF26CDEEFF27CDEEFF34CDE9FF35CDBE
:10199000EAFF1C0EE926000EEA22EF6AA6EC4BF0E5
:1019A00004C00BF005C00CF006C00DF007C00EF02F
:1019B00034CDE9FF35CDEAFF1D0EE926000EEA22FF
:1019C0000BC0EEFF0CC0EEFF0DC0EEFF0EC0EEFF31
:1019D00034CDE9FF35CDEAFF040EEF6E0101000EB4
:1019E000D880D955000EDA551DE234CDE9FF35CD4A
:1019F000EAFF250EE926000EEA22EF8634CDE9FF44
:101A000035CDEAFF120ED9C1EBFF130EDAC1EBFFA1
:101A100034CDE9FF35CDEAFF250EE926000EEA2296
:101A2000EF8402D08CEC2EF002D08CEC2EF001D2A0
:101A300034CDE9FF35CDEAFFEF50030801E07BD05C
:101A4000D7C1E9FFD8C1EAFF0D0EE926000EEA2250
:101A5000EF50020B6DE0242B000E252326232723B5
:101A600034CDE9FF35CDEAFF180EE926000EEA2253
:101A700024CDEEFF25CDEEFF26CDEEFF27CDEEFFE8
:101A8000D7C1E9FFD8C1EAFF0D0EE926000EEA2210
:101A9000EF50100B09E0100E366F34CDE9FF35CD55
:101AA000EAFF040EEF6E1DD0120E366F34CDE9FF43
:101AB00035CDEAFF020EEF6E282B000E29232A23D4
:101AC0002B2334CDE9FF35CDEAFF140EE926000EB5
:101AD000EA2228CDEEFF29CDEEFF2ACDEEFF2BCD59
:101AE000EEFF0101000ED880D955000EDA551DE237
:101AF00034CDE9FF35CDEAFF250EE926000EEA22B6
:101B0000EF8634CDE9FF35CDEAFF120ED9C1EBFFE8
:101B1000130EDAC1EBFF34CDE9FF35CDEAFF250E18
:101B2000E926000EEA22EF8402D08CEC2EF002D0DF
:101B30008CEC2EF07ED1D7C1E9FFD8C1EAFF040EAC
:101B4000E926000EEA22EECF0BF0EECF0CF0EECF3E
:101B50000DF0EFCF0EF034CDE9FF35CDEAFF180ED2
:101B6000E926000EEA220B50EE1809E10C50EE189F
:101B700006E10D50EE1803E10E50EE1800E103E00F
:101B80008CEC2EF08ED134CDE9FF35CDEAFF180E66
:101B9000E926000EEA2224CDEEFF25CDEEFF26CD6C
:101BA000EEFF27CDEEFF34CDE9FF35CDEAFFEF5054
:101BB000040801E0C5D0D7C1E9FFD8C1EAFF0D0E86
:101BC000E926000EEA22EF50100B24E034CDE9FFA5
:101BD00035CDEAFF0F0EEB50FF081CE034CDE9FFD6
:101BE00035CDEAFF0F0EEB500001E26F89EC2EF0CD
:101BF00034CDE9FF35CDEAFF0F0EE926000EEA22CB
:101C0000EF6834CDE9FF35CDEAFF250EE926000E59
:101C1000EA22EF82D7C1E9FFD8C1EAFF0D0EE9261B
:101C2000000EEA22EF50010B31E00D01110E366F6C
:101C300034CDE9FF35CDEAFF140EE926000EEA2285
:101C4000EFCF28FDEE2AEFCF29FDEE22EFCF2AFDC0
:101C5000EE22EFCF2BFDEF2234CDE9FF35CDEAFFA9
:101C6000180EE926000EEA22EF2AEECF24FDEF221D
:101C7000EECF25FDEF22EECF26FDEF22EFCF27FDA1
:101C800034CDE9FF35CDEAFF0A0EEF6E0101000EFB
:101C9000D880D955000EDA5550E234CDE9FF35CD64
:101CA000EAFF250EE926000EEA22EF50080B20E19C
:101CB00034CDE9FF35CDEAFF250EE926000EEA22F4
:101CC000EF8634CDE9FF35CDEAFF120ED9C1EBFF27
:101CD000130EDAC1EBFF34CDE9FF35CDEAFF250E57
:101CE000E926000EEA22EF840D01100E366F24D093
:101CF0000D01366B34CDE9FF35CDEAFF140EE92630
:101D0000000EEA2230CDEEFF31CDEEFF32CDEEFFF8
:101D100033CDEEFF34CDE9FF35CDEAFF180EE926CD
:101D2000000EEA222CCDEEFF2DCDEEFF2ECDEEFFE4
:101D30002FCDEEFF8CEC2EF002D08CEC2EF079D073
:101D400034CDE9FF35CDEAFFEF500A0814E18CEC01
:101D50002EF0D7C1E9FFD8C1EAFF0D0EE926000E2B
:101D6000EA22EF50100B06E034CDD2F135CDD3F19D
:101D7000B6EC0AF05ED034CDE9FF35CDEAFFEF5086
:101D800005083DE18CEC2EF0D7C1E9FFD8C1EAFF90
:101D90000D0EE926000EEA22EF50010B2FE00D0197
:101DA000100E366F34CDE9FF35CDEAFF180EE92667
:101DB000000EEA22EF2AEECF24FDEF22EECF25FD22
:101DC000EF22EECF26FDEF22EFCF27FDD7C1E9FFAF
:101DD000D8C1EAFF0D0EE926000EEA22EF50100BE3
:101DE00007E034CDD2F135CDD3F1B6EC0AF006D010
:101DF00034CDE9FF35CDEAFF060EEF6E1AD034CDB3
:101E0000E9FF35CDEAFFEF50060813E18CEC2EF028
:101E1000D7C1E9FFD8C1EAFF0D0EE926000EEA227C
:101E2000EF50100B06E034CDD2F135CDD3F1B6EC46
:101E30000AF002D08CEC2EF00D013651000831E290
:101E40000101C86BC96B0101C76936CDC6F124CD4C
:101E5000C2F125CDC3F126CDC4F127CDC5F128CDE2
:101E6000BEF129CDBFF12ACDC0F12BCDC1F1D7C133
:101E7000E9FFD8C1EAFFEECFBCF1EDCFBDF1D7C18C
:101E8000E9FFD8C1EAFF020EE926000EEA22EECFF2
:101E9000BAF1EDCFBBF1D5C1B8F1D6C1B9F196EC2D
:041EA00007F0120035
:0C1EA4000001776B03013169326B030110
:101EB0002F6B306BA10E03012D6F2E6BB8EC35F03C
:101EC0000001606F00D012000D01530EA86F4E0E7E
:101ED000A96F4D0EAA6F500EAB6F2E0EAC6F420E57
:101EE000AD6F490EAE6F420EAF6FB06B60C035F391
:101EF00037EC37F0000902E1010E53D060C0B0F0BA
:101F0000E4EC19F000019F0E8D6F0D0E8E6F000135
:101F1000970E8B6F0D0E8C6F92DA0D01A46FA4518A
:101F200001E13BD00001A00E8F6F0D0E906FCBDA58
:101F3000000901E132D0000177910301A80EE86F9A
:101F40000D0EE96F8CEC40F0F3CFA5FDF4CFA6FDAC
:101F50000D01A51D01E1A61D02E000017781A4CDC0
:101F600096F00001A00E946F0D0E956F9FCD93F02B
:101F70000001970E916F0D0E926FD0DA0D01A76FD1
:101F8000000177A102D017EC41F00D01A75101E14A
:101F900004D0ACEC36F0010E04D0BAEC37F0010EF0
:101FA00000D012007AC0E6FF7BC0E6FF610EE66E4D
:101FB000000EE66ED1EC47F0E552E552E552E552EF
:101FC0007CC069F07DC06AF07EC06BF07FC06DF0B0
:101FD00080C06EF081C06FF082C070F078C0CBF32B
:101FE00079C0CCF38FEF4AF00301000ECF6F0D0ED6
:101FF000D06F83C0CDF384C0CEF3A5EC4AF00009C6
:1020000024E083C0E9FF84C0EAFFEECF06FDEECFF7
:1020100007FDEECF08FDEFCF09FDA20E0301316FE2
:10202000326B0301000E2F6F0D0E306F0301FE0E99
:102030002D6F2E69B8EC35F000016C6FFF0E6C5DF2
:1020400002E1000E01D0010E02D0000E00D01200FD
:102050000D01530E346F4E0E356F4D0E366F500E10
:10206000376F2E0E386F420E396F490E3A6F420E9F
:102070003B6F3C6B0301340EE86F0D0EE96F8CEC87
:1020800040F0F3CF32FDF4CF33FD0D01321D01E1FD
:10209000331D06E16CC033F323EC36F0000ECED1D5
:1020A0006CC0B0F0E4EC19F069C000FD0D01610EE8
:1020B000306F000E316F0001300EB16FF5EC19F08A
:1020C00071C026FD72C027FD0001B16BF5EC19F05F
:1020D0000001020EB16FF5EC19F00001010EB16FB5
:1020E000F5EC19F00001B16BF5EC19F00001040EEC
:1020F000B16FF5EC19F000CDB1F0F5EC19F00D0170
:102100000051000700090CE030CDE9FF31CDEAFFB6
:10211000302B000E3123EFCFB1F0F5EC19F0EFD7F3
:102120000001A40EB16FF5EC19F071C028FD72C06A
:1021300029FD0001B16BF5EC19F00001110EB76F2C
:102140000D0EB86F0001010EB56F0D0EB66F0001D8
:10215000140EB36F0D0EB46F6AC0B2F041EC1AF0FA
:10216000000908E117EC41F06CC033F323EC36F0C2
:10217000000E64D10D0117BD08D017EC41F06CC002
:1021800033F323EC36F0000E59D11CCDEAF31DCD0C
:10219000EBF31EEC41F00001060EB16FF5EC19F007
:1021A00032EC41F00D01006F00CD11FD00CDB1F01A
:1021B000F5EC19F00D0100510007000907E032ECC1
:1021C00041F00001B16FF5EC19F0F4D751EC41F09A
:1021D0000001400EB16FF5EC19F00001040EB16F73
:1021E000F5EC19F004C2B1F0F5EC19F005C2B1F04C
:1021F000F5EC19F006C2B1F0F5EC19F007C2B1F038
:10220000F5EC19F00001020EB16FF5EC19F00001C8
:10221000010EB16FF5EC19F00001060EB16FF5EC8F
:1022200019F00001020EB16FF5EC19F00001010E7A
:10223000B16FF5EC19F06BC0B1F0F5EC19F00001DD
:10224000430EB16FF5EC19F00001040EB16FF5EC1F
:1022500019F070C0B1F0F5EC19F06FC0B1F0F5EC09
:1022600019F06EC0B1F0F5EC19F06DC0B1F0F5ECFD
:1022700019F00001300EB16FF5EC19F071C02AFDB4
:1022800072C02BFD0001B16BF5EC19F00001300EAE
:10229000B16FF5EC19F071C02CFD72C02DFD00017D
:1022A000B16BF5EC19F00001100EB76F0D0EB86FA1
:1022B0000001010EB56F0D0EB66F0001140EB36F65
:1022C0000D0EB46F85C0B2F041EC1AF0000908E1C0
:1022D00017EC41F06CC033F323EC36F0000EAED0B7
:1022E0000001060EB16FF5EC19F00D011029000187
:1022F000B16FF5EC19F010CD00FD0D01010E126F5C
:102300000D0E136F0D010051000700090CE012CDF6
:10231000E9FF13CDEAFF122B000E1323EFCFB1F02C
:10232000F5EC19F0EFD78AC0B1F0F5EC19F0000127
:10233000240EC46F0D0EC56F18CDC3F0AEEC1BF0AC
:10234000000908E117EC41F06CC033F323EC36F0E0
:10235000000E74D024CDB1F0F5EC19F0FF0E0D0194
:10236000255D08E117EC41F06CC033F323EC36F047
:10237000000E64D025CD00FD00CDB1F0F5EC19F0D4
:102380000D010051000700090BE00051EA6A860FB9
:10239000E96E000EEA22EFCFB1F0F5EC19F0F0D7BC
:1023A0002529010F1025020F010F006F71C02EFDAE
:1023B00072C02FFD2CCD71F02DCD72F000CDB1F09B
:1023C000F5EC19F0020E0D0100272ACD71F02BCD8E
:1023D00072F000CDB1F0F5EC19F0020E0D01002500
:1023E000060F030F030F060F1125020F006F28CDF4
:1023F00071F029CD72F000CDB1F0F5EC19F0020EBC
:102400000D01002500016925020F030F0D01006F6A
:1024100026CD71F027CD72F000CDB1F0F5EC19F0BA
:102420002ECD71F02FCD72F017EC41F0ACEC36F000
:102430006CC033F323EC36F0010E00D01200000123
:10244000080EAE6F0D0EAF6FC7EC19F0000902E178
:10245000000E38D00001080EA46F0D0EA56FF3EC2E
:1024600018F0000902E1000E2DD00D01085102E024
:10247000000E28D08DC0A2F08EC0A3F08BC0A0F0BB
:102480008CC0A1F0C2EC18F0000902E1000E1AD0D5
:1024900000010C0EA66F0D0EA76F38EC19F00009A5
:1024A00002E1000E0FD08BC04AF28CC04BF20CCD73
:1024B00049F2DEEC21F0000902E1000E03D00D012B
:1024C0000C5100D012000001080EA46F0D0EA56F74
:1024D000F3EC18F0000917E08FC0E9FF90C0EAFFA5
:1024E00008CDEEFF09CDEEFF0ACDEEFF0BCDEEFFDE
:1024F0000001080EA46F0D0EA56FF3EC18F0000993
:1025000004E1000E0AD0000E08D00001080EA46FEE
:102510000D0EA56FF3EC18F000D012000001300E84
:10252000B16FF5EC19F00001820EB16FF5EC19F006
:1025300071C060FD72C061FD0001B16BF5EC19F076
:102540000001B16BF5EC19F00001020EB16FF5EC72
:1025500019F00001010EB16FF5EC19F00001B16B3B
:10256000F5EC19F093C092FD0001040EB16FF5EC8B
:1025700019F093C0B1F0F5EC19F0000193519307F5
:1025800000090CE091C0E9FF92C0EAFF912B000E18
:102590009223EFCFB1F0F5EC19F0EFD70001A20EC6
:1025A000B16FF5EC19F00001820EB16FF5EC19F086
:1025B00071C062FD72C063FD0001B16BF5EC19F0F2
:1025C0000001B16BF5EC19F00001020EB16FF5ECF2
:1025D00019F00001040EB16FF5EC19F094C0E9FF99
:1025E00095C0EAFF030EE926000EEA22EFCFB1F014
:1025F000F5EC19F094C0E9FF95C0EAFF020EE92658
:10260000000EEA22EFCFB1F0F5EC19F094C0E9FF2B
:1026100095C0EAFF010EE926000EEA22EFCFB1F0E5
:10262000F5EC19F094C0E9FF95C0EAFFEFCFB1F0E7
:10263000F5EC19F00001020EB16FF5EC19F0000194
:10264000010EB16FF5EC19F071C064FD72C065FD4B
:102650000001B16BF5EC19F00001020EB16FF5EC61
:1026600019F00001010EB16FF5EC19F071C066FDB3
:1026700072C067FD0001B16BF5EC19F00D015F6BE5
:102680005D6B5E6B0001590EAE6F0D0EAF6FC7EC48
:1026900019F0000902E1000EEAD10001300EB16F1D
:1026A000F5EC19F00001820EB16FF5EC19F071C074
:1026B00068FD72C069FD0001B16BF5EC19F0000115
:1026C000B16BF5EC19F00D01906B916B59515A11EA
:1026D00001E18BD15F2B00015B0EAE6F0D0EAF6F72
:1026E000C7EC19F00D01586F585102E1000EBFD12F
:1026F0005B51595F5C515A5B58510B6E0C6A0B5021
:10270000595F0C505A5B0001300EB16FF5EC19F0B7
:102710000001820EB16FF5EC19F071C06AFD72C054
:102720006BFD0001B16BF5EC19F00001B16BF5EC3C
:1027300019F000017B0EAC6F0D0EAD6F00016C0E39
:10274000AA6F0D0EAB6F93EC19F0000902E1000EB9
:102750008ED1A30E0001965D06E086EC19F000090B
:1027600002E1000E84D10001060EB16FF5EC19F004
:1027700071C093FD72C094FD7BCDB1F0F5EC19F002
:102780000D016C0E7C6F0D0E7D6F7BCD58FD0D0124
:102790005851580700090CE07CCDE9FF7DCDEAFFD8
:1027A0007C2B000E7D23EFCFB1F0F5EC19F0EFD7C5
:1027B00000017E0E9C6F0D0E9D6F7BCD9BF0000186
:1027C0006C0E996F0D0E9A6FCADA000948E10D017F
:1027D000020E5E6F5FCDD2F00001D16F66CDCFF0FB
:1027E00067CDD0F064CDCDF065CDCEF0DDEC1DF041
:1027F000A30E0001965D0FE00001050EB16FF5EC30
:1028000019F00001B16BF5EC19F0040E0D017B25F8
:102810008E6F8F6B23D023EC1AF00001B16FF5ECB3
:1028200019F023EC1AF00D01586F58CDB1F0F5EC0A
:1028300019F0020E0D017B25020F8E6F8F6B0D01BB
:102840005851580700090AE08E2B000E8F2323EC05
:102850001AF00001B16FF5EC19F0F1D7A6D0A00E77
:102860000001965D3EE1020E0D017B258E6F8F6BA0
:1028700071C095FD72C096FD0001CC6B00017E0E0B
:10288000CA6F0D0ECB6F0AEC1DF00D01586F585139
:1028900020E195CD71F096CD72F0020E5E6F5FCDA6
:1028A000D2F00001D16F66CDCFF067CDD0F064CD0E
:1028B000CDF065CDCEF0DDEC1DF00001050EB16F61
:1028C000F5EC19F00001B16BF5EC19F00D01020EF9
:1028D000586F58510B6E0C6A0B508E270C508F237B
:1028E00064D0A10E965D3AE171C095FD72C096FD6F
:1028F00093CD71F094CD72F000017E0E976F0D0EA6
:10290000986FB6D80D01586F585123E195CD71F0ED
:1029100096CD72F05FCDD2F00001020ED16F66CD80
:10292000CFF067CDD0F064CDCDF065CDCEF0DDEC4D
:102930001DF00001050EB16FF5EC19F00001B16B4F
:10294000F5EC19F0020E0D017B25020F8E6F8F6BD7
:1029500004D0020E58258E6F8F6B27D0A30E965D84
:1029600024E100015E0EC86F0D0EC96F00017E0EDE
:10297000C66F0D0EC76FEEEC1BF00D01586F5E5168
:102980000EE05FCDD2F05ECDD1F066CDCFF067CD59
:10299000D0F064CDCDF065CDCEF0DDEC1DF0020EB3
:1029A0000D017B2558258E6F8F6B71C095FD72C010
:1029B00096FD6ACD71F06BCD72F08FCDB1F0F5EC74
:1029C00019F08ECDB1F0F5EC19F0040E0D010C6A82
:1029D0008E250B6E8F510C220B5090270C5091239B
:1029E00095CD71F096CD72F071D668CD71F069CD4C
:1029F00072F091CDB1F0F5EC19F090CDB1F0F5ECAD
:102A000019F0040E0D019025906F000E9121916F29
:102A1000060E9027000E9123030E9027000E91239F
:102A2000030E9027000E912362CD71F063CD72F0FA
:102A300091CDB1F0F5EC19F090CDB1F0F5EC19F0C5
:102A4000050E0D019225040F9025906F000E912127
:102A5000916F60CD71F061CD72F091CDB1F0F5EC78
:102A600019F090CDB1F0F5EC19F0010E00D0120084
:102A70000D01506B006B97C0E9FF98C0EAFF030E91
:102A8000E926000EEA22EF50100B1DE197C0E9FF86
:102A900098C0EAFF030EE926000EEA22EF50040B6D
:102AA000040A01E0010E0B6E97C0E9FF98C0EAFF2F
:102AB000030EE926000EEA22EF50100B100A01E087
:102AC000010E0B140CE00D01010E506F97C09EF02B
:102AD00098C09FF075DA000902E1000E3FD10001B5
:102AE000480EBD6F0D0EBE6F0001150EBB6F0D0EB3
:102AF000BC6F97C0B9F098C0BAF0ADEC1AF00009FD
:102B000002E1000E2BD10D01150E136F0D0E146F87
:102B100071C04CFD72C04DFD48CD00FD010E4C252D
:102B20000001716F000E0D014D210001726F0D014A
:102B30000051000700090CE013CDE9FF14CDEAFFB6
:102B4000132B000E1423EFCFB1F0F5EC19F0EFD7F3
:102B500048CD00FD97C0E9FF98C0EAFF040EEB5096
:102B6000566F97C0E9FF98C0EAFF050EEB504B6F18
:102B700097C0E9FF98C0EAFF030EE926000EEA229B
:102B8000EF50040B3BE10001B16BF5EC19F00D01C6
:102B9000002B71C04EFD72C04FFD4CCD71F04DCD7C
:102BA00072F0482B48CDB1F0F5EC19F04ECD71F034
:102BB0004FCD72F071C04EFD72C04FFD0001CC6B65
:102BC00097C0CAF098C0CBF00AEC1DF00D01026F5F
:102BD000025110E14ECD71F04FCD72F00001050EA3
:102BE000B16FF5EC19F00001B16BF5EC19F00D01C6
:102BF000020E026F025100270051B0D0516B5005F8
:102C000023E10201520E5C6F0D0E5D6F0201510E49
:102C10005A6F0D0E5B6F97C0E9FF98C0EAFF0E0E6A
:102C2000EB500201596F97C0E9FF98C0EAFF050E0B
:102C3000EB500201586F37EC23F0000905E14CCD51
:102C400071F04DCD72F03FD797C0E9FF98C0EAFF11
:102C5000030EE926000EEA22EFCF4AFDE3C3EAF3B2
:102C6000E4C3EBF31EEC41F032EC41F00D01576B85
:102C700032EC41F00D01496F32EC41F00D01086F6B
:102C800032EC41F00D01076F97C0E9FF98C0EAFFF1
:102C90000E0EEB50116F51EC41F00D01505110E14F
:102CA0000201110E566F0D0E576F08CD55F20AEC4A
:102CB00023F0000905E14CCD71F04DCD72F003D742
:102CC0000D010693069906850001010ECC6F0001E7
:102CD000030ECA6F0D0ECB6F0AEC1DF00D015727C6
:102CE00097C0E9FF98C0EAFF0E0E11CDEBFF5751D8
:102CF00000275751482771C04EFD72C04FFD4CCD83
:102D000071F04DCD72F048CDB1F06FDB4ECD71F06A
:102D10004FCD72F097C0E9FF98C0EAFF030EE92695
:102D2000000EEA224ACDEFFF97C0E9FF98C0EAFF04
:102D3000050E4BCDEBFF97C0E9FF98C0EAFF040EEC
:102D400056CDEBFF0001CC6B97C0CAF098C0CBF01A
:102D50000AEC1DF00D010027005100D01200000107
:102D600077B102D0000E2BD10301EF6BF06BACEC0E
:102D700041F0F3CF03FDF4CF04FD9BC005FD03CD6F
:102D8000EAF304CDEBF31EEC41F09CC0E9FF9DC0DB
:102D9000EAFFE3C3EEFFE4C3EDFF32EC41F00D01C7
:102DA000026F32EC41F0E66E9CC0E9FF9DC0EAFF85
:102DB000030EE926000EEA22E552E750EF6E9CC0B2
:102DC000E9FF9DC0EAFF030EE926000EEA22EF505C
:102DD000800B0EE032EC41F0E66E9CC0E9FF9DC036
:102DE000EAFF050EE926000EEA22E552E750EF6EF3
:102DF0009CC0E9FF9DC0EAFF030EE926000EEA220F
:102E0000EF50080B12E032EC41F00D01006F32EC94
:102E100041F00D01016F9CC0E9FF9DC0EAFF0A0E61
:102E200000CDEBFF0B0E01CDEBFF99C0E9FF9AC07F
:102E3000EAFFEF500D01025D22E000019B510D0100
:102E4000055D01E17AD09CC0E9FF9DC0EAFF030E59
:102E5000E926000EEA22EF50080B0DE051EC41F09C
:102E600000CDEFF301CDF0F3ACEC41F0F3CF03FD77
:102E7000F4CF04FD61D051EC41F0000EA0D0050765
:102E80000001992B000E9A239CC0E9FF9DC0EAFF28
:102E9000030EE926000EEA22EF50100B37E19CC02A
:102EA000E9FF9DC0EAFF030EE926000EEA22EF507B
:102EB000010B12E032EC41F00D01006F32EC41F0F9
:102EC0000D01016F9CC0E9FF9DC0EAFF0A0E00CD15
:102ED000EBFF0B0E01CDEBFF32EC41F0E66E9CC038
:102EE000E9FF9DC0EAFF040EE926000EEA22E55242
:102EF000E750EF6E9CC0E9FF9DC0EAFF080EE3C3F8
:102F0000EBFF090EE4C3EBFF18D016D00D01050549
:102F100008E199C0E9FF9AC0EAFFEF5002E10DD045
:102F20000BD0055102E109D007D0E3C303FDE4C390
:102F300004FD51EC41F023D722D751EC41F099C068
:102F4000E9FF9AC0EAFFEFCF02FD9CC0E9FF9DC0F8
:102F5000EAFF0E0E02CDEBFF0D01055113E19CC0FF
:102F6000E9FF9DC0EAFF0E0EE926000EEA22EF6897
:102F70009CC0E9FF9DC0EAFF0F0EE926000EEA2281
:102F8000EF6A1BD00551010803E3800E02150BE028
:102F90009CC0E9FF9DC0EAFF0F0EE926000EEA2261
:102FA000EF680DD00AD09CC0E9FF9DC0EAFF0F0E6C
:102FB000E926000EEA22010EEF6E010E00D012008B
:102FC0009EC0E9FF9FC0EAFF030EE926000EEA2239
:102FD000EF50100B27E19EC0E9FF9FC0EAFF030EF0
:102FE000E926000EEA22EF50080B0BE19EC0E9FF34
:102FF0009FC0EAFF030EE926000EEA22EF50010B04
:103000000FE09EC0E9FF9FC0EAFF0A0EE926000E0E
:10301000EA22EECFEFF3EDCFF0F3ACEC41F002D0CB
:10302000000EAFD09EC0E9FF9FC0EAFFE3C3EEFFF2
:10303000E4C3EDFF9EC0E9FF9FC0EAFFEECFEAF3D5
:10304000EDCFEBF31EEC41F032EC41F0E66E9EC0AA
:10305000E9FF9FC0EAFF020EE926000EEA22E552D0
:10306000E750EF6E32EC41F0E66E9EC0E9FF9FC084
:10307000EAFF030EE926000EEA22E552E750EF6E62
:103080009EC0E9FF9FC0EAFF030EE926000EEA2278
:10309000EF50800B0EE032EC41F0E66E9EC0E9FF8F
:1030A0009FC0EAFF050EE926000EEA22E552E7502E
:1030B000EF6E9EC0E9FF9FC0EAFF030EE926000EF7
:1030C000EA22EF50080B0BE19EC0E9FF9FC0EAFF28
:1030D000030EE926000EEA22EF50010B12E032EC5B
:1030E00041F00D01B16F32EC41F00D01B26F9EC0A5
:1030F000E9FF9FC0EAFF0A0EB1CDEBFF0B0EB2CD88
:10310000EBFF9EC0E9FF9FC0EAFF030EE926000E19
:10311000EA22EF50100B03E051EC41F083D732EC80
:1031200041F0E66E9EC0E9FF9FC0EAFF040EE9266B
:10313000000EEA22E552E750EF6E9EC0E9FF9FC005
:10314000EAFF080EE3C3EBFF090EE4C3EBFF9EC0EA
:10315000E9FF9FC0EAFF0F0EE926000EEA22010EEA
:10316000EF6E9EC0E9FF9FC0EAFF0E0EE926000E3B
:10317000EA22EF6A51EC41F0010E03D053D7000E62
:1031800000D0120060D90D01006F040E005D02E056
:10319000000E28D058D90D01016FA2C0E9FFA3C0CD
:1031A000EAFF01CDEFFF0151080802E2000E1AD03C
:1031B0000D010151010700090EE045D90D01006F15
:1031C0000001A0C0E9FFA1C0EAFFA02B000EA123CF
:1031D00000CDEFFFEDD7A0C0E9FFA1C0EAFFEF6A85
:1031E000010E00D012000D01046B056B066B076B1E
:1031F0002AD9020802E0000E3AD00001040EA86F9E
:103200000D0EA96F51D8000902E1000E30D0040E56
:10321000D8800D010455000E0555000E0655000E10
:10322000075502E2000E23D0006B016B026B036BAB
:103230000451040700090DE006D9E66E0D010451A2
:10324000EA6A000FE96E0D0EEA22E552E750EF6ED2
:10325000EFD7A4C0E9FFA5C0EAFF00CDEEFF01CD86
:10326000EEFF02CDEEFF03CDEEFF010E00D0120007
:10327000EAD80D01006FA00E005D08E0A10E005D10
:1032800005E0A30E005D02E0000E0DD0A6C0E9FF30
:10329000A7C0EAFF00CDEFFF0001010EA86F0D0EE1
:1032A000A96F02D800D012000D010E6B0F6B106BCE
:1032B000CAD80D010D6F0DCD0EFD0DAF1AD00D9FAB
:1032C0000D51020802E2000E20D00D29106F0D51A1
:1032D0000D0700090DE0B7D8E66E0D010D51EA6A41
:1032E0000E0FE96E0D0EEA22E552E750EF6EEFD7B2
:1032F00002D0010E106FA8C0E9FFA9C0EAFF0ECDF1
:10330000EEFF0FCDEDFF105100D012009CD8050844
:1033100002E0000E07D097D8000902E0000E01D0AD
:10332000010E00D012008FD8060802E0000E2ED049
:103330000001000EA86F0D0EA96FB6DF000902E1B3
:10334000000E24D00D010F0ED8800055000E01553F
:1033500002E2000E1BD0ACC0E9FFADC0EAFF00CD19
:10336000EFFF0D010051000700090EE06CD8E66E7A
:103370000001AAC0E9FFABC0EAFFAA2B000EAB23F5
:10338000E552E750EF6EEDD7010E00D012005BD88A
:10339000300802E0000E17D00001000EA86F0D0EDD
:1033A000A96F82DF0D01046F045102E1000E0BD002
:1033B000042BAEC0E9FFAFC0EAFF00CDEEFF01CDA8
:1033C000EDFF045100D01200B0C02CF3B3EC2DF08F
:1033D000000901E1F9D7D6C075F0D7C076F0000139
:1033E000736B746B716B726B120003012C51160DB1
:1033F000F3CFE9FFF4CFEAFF000EE926030EEA223D
:10340000130EE926000EEA2271C0EEFF72C0EDFF36
:10341000080E000171250001F26F000E00017221FB
:103420000001F36F140EF227000EF32376C0F1F0C3
:1034300037EC30F0B1C034F335EC36F00001712BCD
:10344000000E72231200000173C0EFF074C0F0F0A0
:10345000732B000E7423080E0001EF27000EF023DB
:10346000140EEF27000EF0230CEC30F00301110EC8
:10347000366F0D0E376F52EC37F00D01115100D041
:1034800012000301EF6BF06BACEC41F0F3CF45FDA4
:10349000F4CF46FDB3C0C1F0B4C0C2F045CDBFF01B
:1034A00046CDC0F0C9D8B3C0E9FFB4C0EAFF030EEF
:1034B000E926000EEA22EF50100B49E1B3C0E9FF04
:1034C000B4C0EAFF030EE926000EEA22EF50800B9B
:1034D00017E0B3C0E9FFB4C0EAFF050EEB500001EE
:1034E000B25D0EE1B7C0BDF0B8C0BEF0B5C0BBF074
:1034F000B6C0BCF0B3C0B9F0B4C0BAF02ED82CD06E
:10350000B3C0E9FFB4C0EAFF030EE926000EEA22C9
:10351000EF50080B0BE1B3C0E9FFB4C0EAFF030EA4
:10352000E926000EEA22EF50010B0FE0B3C0E9FFDD
:10353000B4C0EAFF0A0EE926000EEA22EECFEFF34E
:10354000EDCFF0F3ACEC41F002D0000E05D0E3C3B8
:1035500045FDE4C346FD9ED712000301EF6BF06BFF
:10356000ACEC41F0F3CFB3FDF4CFB4FDB9C0E9FF4B
:10357000BAC0EAFFEECFB1FDEDCFB2FD0D01C86BD1
:10358000C76B0001B70EC16F0D0EC26FB3CDBFF098
:10359000B4CDC0F051D80D01C7510001EA6ABB2576
:1035A000E96EBC51EA22B9CDEFFF0D01B351B1195B
:1035B00002E1B451B21909E1C72BBDC0E9FFBEC099
:1035C000EAFFC7CDEFFF010E36D0C851010A24E053
:1035D000010A01E02DD0BAB703D0010EC86F1CD08C
:1035E000C1CDB5FDC2CDB6FDB5CDEFF3B6CDF0F38F
:1035F000ACEC41F0E3C3B5FDE4C3B6FD0D01B5513C
:10360000B15DB651B25906E3B5CDB3FDB6CDB4FD4B
:103610000FD002D0010EC86F0D01BAB902D0000E52
:103620000AD0C72BC3CDB3FDC4CDB4FDC86B00D049
:10363000A8D7000E00D01200BFC0EAF3C0C0EBF361
:103640001EEC41F0C1C0E9FFC2C0EAFFBFC0EEFFFF
:10365000C0C0EDFF32EC41F0E66EC1C0E9FFC2C070
:10366000EAFF020EE926000EEA22E552E750EF6E6D
:1036700032EC41F0E66EC1C0E9FFC2C0EAFF030EC2
:10368000E926000EEA22E552E750EF6EC1C0E9FFDD
:10369000C2C0EAFF030EEB500D01C96FC9AF0ED0D7
:1036A00032EC41F0E66EC1C0E9FFC2C0EAFF050E90
:1036B000E926000EEA22E552E750EF6E0D01C9A798
:1036C00012D032EC41F00D01CA6F32EC41F00D0125
:1036D000CB6FC1C0E9FFC2C0EAFF0A0ECACDEBFF43
:1036E0000B0ECBCDEBFFC9A90BD0C1C0E9FFC2C007
:1036F000EAFF0C0EE3C3EBFF0D0EE4C3EBFF2CD08F
:10370000C9A112D032EC41F00D01CA6F32EC41F088
:103710000D01CB6FC1C0E9FFC2C0EAFF0A0ECACDDE
:10372000EBFF0B0ECBCDEBFF32EC41F0E66EC1C0F0
:10373000E9FFC2C0EAFF040EE926000EEA22E552C4
:10374000E750EF6EC1C0E9FFC2C0EAFF080EE3C355
:10375000EBFF090EE4C3EBFF51EF41F00A0E00014D
:10376000E76EC319E8AE02D0E73402D0E750C35D7C
:1037700002E3000E32D0C3C0F6FFF76AF6BEF76868
:10378000D890F636F736DA0EF626970EF7220800AE
:10379000F550E66EC4C0E9FFC5C0EAFFE552E75048
:1037A000EF6EC3C0F6FFF76AF6BEF768D890F6363C
:1037B000F736DA0EF626970EF722F62A000EF722D3
:1037C0000800F550E66EC4C0E9FFC5C0EAFFEE523E
:1037D000E552E750EF6E010E00D012000D01006BB4
:1037E0000B6BC6C0E9FFC7C0EAFF030EE926000E57
:1037F000EA22EF50100B16E1C6C0E9FFC7C0EAFF8E
:10380000030EE926000EEA22EF50020B0BE1C6C0C0
:10381000E9FFC7C0EAFF030EE926000EEA22EF50D7
:10382000200B02E1020E006F0EDE0D01036F03CDCF
:10383000B1F0DBDD0D010B2B0001010EC46F0D0E8D
:10384000C56FC6C0E9FFC7C0EAFF040EEB50000118
:10385000C36F84DF000903E10D01030E006F0D014A
:103860000151035D02E0030E006FEDDD0D01046FF9
:1038700004CDB1F0BADD0D010B2B04517F0802E23B
:10388000030E006FC6C0E9FFC7C0EAFF030EE926BA
:10389000000EEA22EF50040B0AE1C6C0E9FFC7C0E0
:1038A000EAFF0E0EEB50000902E0020E006F056BFE
:1038B000066B076B086B096BFF0E025D3FE004515E
:1038C000040839E304510407000911E0BCDD0D01CF
:1038D0000A6F0451EA6A050FE96E0D0EEA220ACD5D
:1038E000EFFF0ACDB1F081DD0D010B2BEBD70051BD
:1038F00021E105CD51F206CD52F207CD53F208CDAC
:1039000054F209CD50F2C6C0E9FFC7C0EAFF0E0E5F
:10391000EB5002014F6FC6C0E9FFC7C0EAFF050EBA
:10392000EB5002014E6FF7EC21F0000903E10D01AD
:10393000030E006F02D0030E006F62D004CD4DF273
:10394000C6C0E9FFC7C0EAFF050EEB5002014C6F8D
:10395000E1EC21F0000903E10D01030E006F0D0100
:103960000451040700092EE06EDD0D01056F05CD41
:10397000B1F03BDD0D010B2B005123E105CD51F2E0
:1039800006CD52F207CD53F208CD54F20951092B5E
:103990000201506FC6C0E9FFC7C0EAFF0E0EEB5030
:1039A00002014F6FC6C0E9FFC7C0EAFF050EEB502A
:1039B00002014E6FF7EC21F0000903E10D01030E47
:1039C000006FCDD700511CE105CD51F206CD52F26A
:1039D00007CD53F208CD54F202015069C6C0E9FF89
:1039E000C7C0EAFF0E0EEB5002014F6FC6C0E9FFE1
:1039F000C7C0EAFF050EEB5002014E6FF7EC21F055
:103A0000C8C0E9FFC9C0EAFF00CDEFFF0D010B51AF
:103A100000D012000D01C76BC86BC96BCA6BCAC05E
:103A2000E9FFCBC0EAFF030EE926000EEA22EF50C1
:103A3000100B02E0000EC0D0CAC0E9FFCBC0EAFF05
:103A4000030EE926000EEA22EF50040B0AE1CAC079
:103A5000E9FFCBC0EAFF0E0EEB50000802E2000EB9
:103A6000ABD0CAC0E9FFCBC0EAFF040EEB50CC6F6D
:103A70000001CD0EC46F0D0EC56FCCCDC3F06EDE50
:103A8000000902E1000E98D00001CC510AE1CDCD31
:103A9000B1F0ABDC71C0CFFD72C0D0FDCECDB1F0C6
:103AA000A4DCCAC0E9FFCBC0EAFF030EE926000E82
:103AB000EA22EF50020B22E0CAC0E9FFCBC0EAFFC6
:103AC000080EE926000EEA22EECFEAF3EDCFEBF383
:103AD0001EEC41F032EC41F00D01CB6FCBCDC6FDB9
:103AE0000D01C651C607000906E032EC41F00001A5
:103AF000B16F7BDCF5D751EC41F046D00D01C56BC1
:103B0000C76BC86BC96BCA6BCB6B0201C70E5C6F0E
:103B10000D0E5D6F0201C50E5A6F0D0E5B6FCAC0B0
:103B2000E9FFCBC0EAFF0E0EEB500201596FCAC08D
:103B3000E9FFCBC0EAFF050EEB500201586F37ECEE
:103B400023F000091FE0FF0E0D01CE5D12E0CECD87
:103B5000CBFD0D01CE510BE0CE07CE51EA6AC70F67
:103B6000E96E0D0EEA22EFCFB1F03FDCF2D70CD0B8
:103B700004D0CB2BC7CDB1F038DCFF0E0D01C55DF5
:103B8000C4E102D0000E18D00001CC5112E171C086
:103B9000D1FD72C0D2FDCFCD71F0D0CD72F0CBCDC2
:103BA000B1F023DCD1CD71F0D2CD72F00D01CB2B71
:103BB000CB2B0D01CB5100D0120071C000FD72C0A3
:103BC00001FDCDC071F0CEC072F0D1C0B1F00DDCFE
:103BD000CFC071F0D0C072F0D2C0B1F0F5EC19F0E6
:0A3BE00000CD71F001CD72F012006B
:063BEA00DACFE4FFE2CF98
:103BF000DAFFE9CFE4FFEACFE4FF00EE0BF0080EB6
:103C0000E80403E3EECFE4FFFBD7E652B7EC4BF05A
:103C1000E55200EE12F0080EE80403E3E5CFEDFFF5
:103C2000FBD7E5CFEAFFE5CFE9FFE5CFDAFF1100EB
:103C3000ACA2FED721C2ADFF1200020122C2E9FFF1
:103C400023C2EAFF222B000E2323EFCF08FDEF5003
:103C500004E008CD21F2ECDFF0D7120086EC24F06E
:103C60009DEC4BF081EC40F0B4EC24F081BA0ED026
:103C70000401C00E256FAFEC49F00401DB0E286F84
:103C80008C0E296F06EC4AF0C9EC26F027EC44F0C4
:103C9000C1EC27F026EC39F052EC0FF002011CA128
:103CA0000DD00401C00E256FAFEC49F00401CA0E1F
:103CB000286F8C0E296F06EC4AF006D00201010E27
:103CC000E36F0201070EFB6FA6EC4BF00201E4511B
:103CD000045C0B6EE55105580C6EE65106580D6EEE
:103CE000E75107580E6E320E0B5C000E0C58000E9A
:103CF0000D58000E0E580BE3A6EC4BF004C0E4F296
:103D000005C0E5F206C0E6F207C0E7F2897832ECBA
:103D100044F0EDEC27F035EC39F064EC0FF0EFD81F
:103D20000201E3510201FE5D24E00201010E266F53
:103D30000201040E246F020E256F1DD8FEC2E3F2AD
:103D400002011CA116D00401CE0E256FAFEC49F084
:103D50000A0E0201E35D07E2300EE32504012A6F3B
:103D600018EC4AF006D0410EE32504012A6F18EC46
:103D70004AF0AAD71200020126510CE00401C00E3D
:103D8000256FAFEC49F00401EA0E286F8C0E296F05
:103D900006EC4AF00401C00E256FAFEC49F0000EAE
:103DA000E66E0D0EE66E24C2E9FF25C2EAFFEF5073
:103DB000E66EE66ABCEC45F0E552E552E552E552A6
:103DC000020126510DE00401000E266F0D0E276F33
:103DD000F5EC49F004012E0E2A6F18EC4AF00AD0D7
:103DE0000201000E226F0D0E236F27DF02012E0E3F
:103DF000216F1EDF000EE66E0D0EE66E24C2E9FF97
:103E000025C2EAFF010EE926000EEA22EF50E66E17
:103E1000E66ABCEC45F0E552E552E552E552020196
:103E200026510DE00401000E266F0D0E276FF5ECF4
:103E300049F004012E0E2A6F18EC4AF00AD0020154
:103E4000000E226F0D0E236FF8DE02012E0E216F81
:103E5000EFDE000EE66E0D0EE66E24C2E9FF25C20F
:103E6000EAFF020EE926000EEA22EF50E66EE66A4D
:103E7000BCEC45F0E552E552E552E552020126510F
:103E80000DE00401000E266F0D0E276FF5EC49F0D2
:103E900004012E0E2A6F18EC4AF00AD00201000E1F
:103EA000226F0D0E236FC9DE02012E0E216FC0DEC0
:103EB000000EE66E0D0EE66E24C2E9FF25C2EAFF93
:103EC000030EE926000EEA22EF50E66EE66ABCEC2D
:103ED00045F0E552E552E552E5520201265108E06F
:103EE0000401000E266F0D0E276FF5EC49F006D089
:103EF0000201000E226F0D0E236F9FDE1200815013
:103F0000200B05E10201E85102E1010EE86F020118
:103F1000C651E95D02E1E96BE86BE85127E0E95140
:103F20000E0DF3CFE9FFF4CFEAFFC70EE926020E2C
:103F3000EA220D0EE926000EEA22EF50010B15E0F1
:103F40000D01416B41CD45F242CD46F243CD47F2E2
:103F500044CD48F20201070E446FE9C243F286D90C
:103F6000000902E00201E92B01D0E92B810EC26EAB
:103F70000201640E006F00510007000901E0FBD749
:103F8000C282C2B2FED7C3CF00F2C4CF01F2270E65
:103F9000E66E020EE66E00C2E6FF01C2E6FFBCEC72
:103FA00045F0E552E552E552E5520D0EC16E890E1F
:103FB000C26E0201640E026F02510207000901E0A5
:103FC000FBD7C282C2B2FED7C3CF02F2C4CF03F284
:103FD0002F0EE66E020EE66E02C2E6FF03C2E6FF99
:103FE000BCEC45F0E552E552E552E5528E0EC16E4D
:103FF000120037C2E9FF38C2EAFFEE50EFCFEAFF06
:10400000E96EEF50D00F0D01656F6551010A55E063
:10401000010A1DE00A0EE66EE66A080E0B6E8D0EB2
:104020000C6E0D6A0BC0E6FF0CC0E6FF0DC0E6FF8C
:1040300037C2E9FF38C2EAFFEECFE6FFEFCFE6FF77
:10404000AEEC47F0F56E070EE15EF55037D0020E8C
:104050000201EA6A3725E96E3851EA22EE50EFCFC5
:10406000EAFFE96EEF50D00F0D01666F6651010A4D
:1040700005E0010A01E004D0897602D0897400D0FD
:104080000D0EE66EE66AFB0E0B6E8C0E0C6E0D6A64
:104090000BC0E6FF0CC0E6FF0DC0E6FF37C2E9FF2C
:1040A00038C2EAFFEECFE6FFEFCFE6FFAEEC47F017
:1040B000F56E070EE15EF55001D000D0120002014E
:1040C0003A51040A01E181D0070A53E0010A25E0D0
:1040D000030A13E0010A01E088D089A607D0300E58
:1040E0003DC2E9FF3EC2EAFFEF6E06D0310E3DC28F
:1040F000E9FF3EC2EAFFEF6E78D089A407D0300E08
:104100003DC2E9FF3EC2EAFFEF6E06D0310E3DC26E
:10411000E9FF3EC2EAFFEF6E68D03B513C1102E17D
:104120003B6B3C6B3B51EA6A270FE96E020EEA22B9
:10413000EF503DC2E9FF3EC2EAFFEF6E3B51EA6A33
:10414000270FE96E020EEA22EF5007E10B680C68B8
:104150000BC0F3FF0CC0F4FF4FD03BC20BF03CC2CE
:104160000CF03B2B000E3C233BC2F3FF3CC2F4FFA0
:1041700043D03B513C1102E13B6B3C6B3B51EA6A43
:104180002F0FE96E020EEA22EF503DC2E9FF3EC258
:10419000EAFFEF6E3B51EA6A2F0FE96E020EEA2248
:1041A000EF5007E10B680C680BC0F3FF0CC0F4FF85
:1041B00023D03BC20BF03CC20CF03B2B000E3C2347
:1041C0003BC2F3FF3CC2F4FF17D081AA07D0310EE7
:1041D0003DC2E9FF3EC2EAFFEF6E06D0300E3DC29F
:1041E000E9FF3EC2EAFFEF6E00D00B680C680BC01F
:1041F000F3FF0CC0F4FF00D01200030EE66EE66A77
:10420000120E0B6E8D0E0C6E0D6A0BC0E6FF0CC00D
:10421000E6FF0DC0E6FF3FC2E6FF40C2E6FF64ECEA
:1042200047F0F56E070EE15EF55000091CE1090E3E
:10423000E66EE66A160E0B6E8D0E0C6E0D6A0BC0E6
:10424000E6FF0CC0E6FF0DC0E6FF41C2E6FF42C23A
:10425000E6FF64EC47F0F56E070EE15EF5500009ED
:1042600002E1010E02D0000E00D012000201435103
:104270000E0DF3CFE9FFF4CFEAFFC70EE926020ED9
:10428000EA22090EE926000EEA22030EE926000EB4
:10429000EA22EFCF3DFD43510E0DF3CFE9FFF4CFFE
:1042A000EAFFC70EE926020EEA22090EE926000EF1
:1042B000EA22020EE926000EEA22EFCF3EFD43512C
:1042C0000E0DF3CFE9FFF4CFEAFFC70EE926020E89
:1042D000EA22090EE926000EEA22010EE926000E66
:1042E000EA22EFCF3FFD43510E0DF3CFE9FFF4CFAC
:1042F000EAFFC70EE926020EEA22090EE926000EA1
:10430000EA22EFCF40FD0201EA51010A39E0010A39
:1043100001E051D0A6EC4BF004C07FF005C080F066
:1043200006C081F007C082F00001060E7E6F00011A
:104330007D69020143510E0DF3CFE9FFF4CFEAFF8F
:10434000C70EE926020EEA22EFCF7CF043510E0D94
:10435000F3CFE9FFF4CFEAFFC70EE926020EEA2207
:10436000EE52E9CF7AF0EACF7BF000013D0E786F94
:104370000D0E796FD2EC0FF00201010EEA6F1BD027
:1043800000013D0E836F0D0E846FF4EC0FF00009F9
:1043900012E00201EA6B00018A6B45C286F046C258
:1043A00087F047C288F048C289F044C285F028EC03
:1043B00010F0010E02D0000E00D01200010E00D04D
:1043C000120002014C510A0A09E00E0A01E00CD069
:1043D000090E4D5D02E2010E09D006D0110E4D5DB1
:1043E00002E2010E03D000D0000E00D01200020144
:1043F0004E510A0A01E1EFD00E0A01E1A7D0060AE8
:1044000065E0010A1CE0050A0EE0030A01E0FFD0A6
:104410005151010BF36EF346F346FB0E8914F31072
:10442000896E010EF6D05151010BF36EF346F3463F
:10443000F346F70E8914F310896E010EEAD00201DB
:10444000C65102014F5D19E24F510E0DF3CFE9FF46
:10445000F4CFEAFFC70EE926020EEA22090EE9268A
:10446000000EEA2251C2EEFF52C2EEFF53C2EEFF2F
:1044700054C2EEFF010ECDD028D0020E4F5D25E2D2
:104480004F510E0DF3CFE9FFF4CFEAFFC70EE92637
:10449000020EEA22090EE926000EEA2251C2EEFFC0
:1044A00052C2EEFF53C2EEFF54C2EEFF4F510E0D4B
:1044B000F3CFE9FFF4CFEAFFC70EE926020EEA22A6
:1044C000EF6A0201C62B010EA4D0A1D00201C65191
:1044D00002014F5D29E2510510E14F510E0DF3CF5E
:1044E000E9FFF4CFEAFFC70EE926020EEA220D0E1D
:1044F000E926000EEA22EF8014D0515110E14F510D
:104500000E0DF3CFE9FFF4CFEAFFC70EE926020E46
:10451000EA220D0EE926000EEA22EF9002D0000EEC
:1045200078D0010E76D011D0020E4F5D0EE202015E
:10453000C62B02014F510E0DF3CFE9FFF4CFEAFF76
:10454000C70EE926020EEA22EF6A61D0FF0E505D27
:1045500015E10201C65102014F5D02E10201C62BC5
:1045600002014F510E0DF3CFE9FFF4CFEAFFC70E62
:10457000E926020EEA22EF2A010E4BD00201C651B3
:1045800002014F5D27E24F510E0DF3CFE9FFF4CF4B
:10459000EAFFC70EE926020EEA22EE52E9CF0BF03F
:1045A000EACF0CF050510F010B24E96F000E0C20E4
:1045B000EA6F51C2EFFF02014F510E0DF3CFE9FF39
:1045C000F4CFEAFFC70EE926020EEA2250C2EFFF3F
:1045D000010E1FD01CD0FF0E505D0BE05051EA6A57
:1045E000B50FE96E020EEA2251C2EFFF0201C52BA0
:1045F0000CD00401800E256FAFEC49F00401B50E1C
:10460000266F020E276FF5EC49F0010E02D0000E66
:1046100000D0120056C2E9FF57C2EAFFEFCFB1FD4A
:1046200002015551010A01E01FD00201C65102E109
:10463000000E1CD0FF0E0D01B15D08E156C2E9FF6E
:1046400057C2EAFFEF6A010E11D00DD00201C60574
:104650000D01B15D08E2B12956C2E9FF57C2EAFF78
:10466000EF6E010E03D000D0000E00D012005AC22F
:10467000E9FF5BC2EAFFEFCFB1FD020158510A0A20
:1046800001E11CD10E0A01E1C2D0070A01E195D077
:10469000010A73E0030A63E0080A57E0010A4BE0ED
:1046A0000F0A3BE0010A2BE0030A1BE0FF0A01E0CE
:1046B0002AD1A6EC4BF004C00BF005C00CF006C0EC
:1046C0000DF007C00EF05CC2E9FF5DC2EAFF0BC04F
:1046D000EEFF0CC0EEFF0DC0EEFF0EC0EEFF010EB0
:1046E00014D18950040B01E0010EE66E5CC2E9FFB3
:1046F0005DC2EAFFE552E750EF6E010E06D1895028
:10470000080B01E0010EE66E5CC2E9FF5DC2EAFF44
:10471000E552E750EF6E010EF8D08150200B01E01A
:10472000010EE66E5CC2E9FF5DC2EAFFE552E750AA
:10473000EF6E010EEAD05CC2E9FF5DC2EAFF00C283
:10474000EEFF01C2EDFF010EE0D05CC2E9FF5DC2E9
:10475000EAFF02C2EEFF03C2EDFF010ED6D0020156
:10476000C6510201595D08E25CC2E9FF5DC2EAFF81
:1047700059C2EFFF010EC9D0C6D00201C6510201D5
:10478000595D1AE259510E0DF3CFE9FFF4CFEAFF5C
:10479000C70EE926020EEA220D0EE926000EEA22D5
:1047A000EF50010BE66E5CC2E9FF5DC2EAFFE55225
:1047B000E750EF6E010EA9D0A6D00201C65102014A
:1047C000595D24E259510E0DF3CFE9FFF4CFEAFF12
:1047D000C70EE926020EEA22090EE926000EEA2299
:1047E000EECF0BF0EECF0CF0EECF0DF0EFCF0EF0E2
:1047F0005CC2E9FF5DC2EAFF0BC0EEFF0CC0EEFF3A
:104800000DC0EEFF0EC0EEFF010E7FD07CD0020186
:10481000C6510201595D51E259510E0DF3CFE9FF26
:10482000F4CFEAFFC70EE926020EEA22EF5006E1B6
:104830005AC2E9FF5BC2EAFFEF683DD059510E0D45
:10484000F3CFE9FFF4CFEAFFC70EE926020EEA2212
:10485000EE52E9CF0BF0EACF0CF00D01B1510F0190
:104860000B24E96F000E0C20EA6FEF50E66E5CC27D
:10487000E9FF5DC2EAFFE552E750EF6E0D01B12B93
:10488000020159510E0DF3CFE9FFF4CFEAFFC70E35
:10489000E926020EEA22EF500D01B15D06E15AC28F
:1048A000E9FF5BC2EAFFEF6806D05AC2E9FF5BC2CC
:1048B000EAFFB1CDEFFF010E28D025D00201C5518E
:1048C00003E10D01B16917D00D01B151B12BEA6AB5
:1048D000B50FE96E020EEA22EF50E66E5CC2E9FF08
:1048E0005DC2EAFFE552E750EF6E0201C5510D01CE
:1048F000B15D01E1B1695AC2E9FF5BC2EAFFB1CD26
:10490000EFFF010E02D0000E00D012008E0EC16E1D
:10491000030E926E020EC06E809A89848986F19E83
:1049200069EC49F00401800E256FAFEC49F00401F9
:10493000AC0E286F8C0E296F06EC4AF00401C00EF5
:10494000256FAFEC49F00401BA0E286F8C0E296F69
:1049500006EC4AF0200EAC6E900EAB6E0F0EAF6EF2
:10496000D56AF28EF28C120002010A0E046F056FF6
:10497000050E066F0F0E076F0E690F691069116B38
:104980000A0E126F136F050E146F0F0E156F086B62
:10499000040E096FA30E0A6F0B6B0C6B0D6B1C8161
:1049A0000D01040E046F020E056F0301D66BD76B69
:1049B0000301A00ED56F73EC3FF0E4EC3FF00D0166
:1049C000036FEEEC3FF0550E0D01035D26E1010E85
:1049D0000301D66FD76B0301A00ED56F73EC3FF0C8
:1049E0000D01036B03510B6E0C6A1D0E0B5C000E68
:1049F0000C5810E2E4EC3FF0E66E0D0104CDE9FF47
:104A000005CDEAFF042B000E0523E552E750EF6EBB
:104A1000032BE8D7EEEC3FF001D001D812000D01D6
:104A2000040E016F020E026F0301D36BD46B0301FE
:104A3000A00ED26F1FEC3FF00301550ED86FB2EC01
:104A40003FF00D01006B00510B6E0C6A1D0E0B5CEC
:104A5000000E0C580EE201CDE9FF02CDEAFF012B5A
:104A6000000E0223EFCFD8F3B2EC3FF00D01002B84
:104A7000EAD7D4EF3FF002015EC2F6FF5FC2F7FF54
:104A80005E2B000E5F230800F5CF00FDF55005E01A
:104A900000CD21F218EC1EF0EED712000D01016BD3
:104AA0009EAAFED7AECF00FD0D0E0D01005D03E006
:104AB0000A0E005D01E116D0012B020160C2E9FF80
:104AC00061C2EAFF602B000E612300CDEFFF60C2E0
:104AD000E9FF61C2EAFFEF6A62516207000901E182
:104AE00001D0DED70D01015100D0120063C201FDDB
:104AF00064C202FD0D01036B63C2E9FF64C2EAFFF9
:104B0000EFCF00FDEF503DE02E0E0D01005D2CE1DA
:104B1000020163C2E9FF64C2EAFF632B000E642353
:104B2000EF6A01CDE6FF02CDE6FF47EC45F0E55226
:104B3000E552F350E66E65C2E9FF66C2EAFFE9CFCF
:104B40000BF0EACF0CF00D010351032B0F010B24E6
:104B5000E96F000E0C20EA6FE552E750EF6E63C27A
:104B600001FD64C202FD08D0300E005D03E3005178
:104B7000390802E2000E2AD00201632B000E6423E2
:104B8000BBD701CDE6FF02CDE6FF47EC45F0E5528D
:104B9000E552F350E66E65C2E9FF66C2EAFFE9CF6F
:104BA0000BF0EACF0CF00D0103510F010B24E96F5C
:104BB000000E0C20EA6FE552E750EF6E030E0D0178
:104BC000035D02E0000E01D0010E00D012009EAA8B
:104BD000FED7AECF00FD310E0D01005D06E3390EAC
:104BE000005D03E2005103D002D0390E00D0120064
:104BF00002010D0E216F18EC1EF002010A0E216F4A
:104C000018EC1EF0300E0201675DFF0FE96EEA6AD4
:104C1000D890E936EA36EB0EE926020EEA22EECF0C
:104C20005EF2EDCF5FF227DF02016751380A01E142
:104C3000ADD00F0A01E1A8D0010A01E1A3D0030A17
:104C400001E19ED0010A54E0070A4CE0010A44E069
:104C5000030A01E09DD08F0EE66E0D0EE66E16C2C1
:104C6000E6FF17C2E6FFBCEC45F0E552E552E5521F
:104C7000E55202018F0E226F0D0E236F1DEC1EF008
:104C80000201290E216F18EC1EF002013A0E216F6D
:104C900018EC1EF00201200E216F18EC1EF002012C
:104CA000140E626F02018F0E606F0D0E616FF6DEE3
:104CB000000911E08F0EE66E0D0EE66E47EC45F032
:104CC000E552E552F3CF16F2F4CF17F217C20CF209
:104CD00016C20DF25DD03ED00D01040EA76F020E7C
:104CE000A86F0BD00D01120EA76F020EA86F05D092
:104CF0000D010E0EA76F020EA86F0201266BA7CD45
:104D000024F2A8CD25F2BBEC1EF00201290E216F82
:104D100018EC1EF002013A0E216F18EC1EF0020191
:104D2000200E216F18EC1EF00201140E626F0201BA
:104D30008F0E606F0D0E616FB1DE0201A30E656F05
:104D40000D0E666F02018F0E636F0D0E646FCEDE67
:104D5000000909E102017D0E5E6F8E0E5F6F8BDE32
:104D60009EAAFED70CD0A7CDE9FFA8CDEAFFA3CD20
:104D7000EEFFA4CDEEFFA5CDEEFFA6CDEEFF08D051
:104D80001C8106D01C9104D018D802D048DE00D077
:104D900012000201200E5E6F8D0E5F6F6CDE17DF5A
:104DA0000D01AA6F390EAA5D03E0AACD67F220DFDC
:104DB000380E0D01AA5DEDE112000D01006B046BD0
:104DC00059EC41F0F3CF02FDF4CF03FDA6EC4BF01C
:104DD00004C087FD05C088FD06C089FD07C08AFDA7
:104DE000B7EC4BF0A6EC4BF004C08BFD05C08CFD7E
:104DF00006C08DFD07C08EFD870EE96E0D0EEA6EB2
:104E0000EE500D018B5D0B6EEE508C590C6EEE501A
:104E10008D590D6EEE508E590E6E320E0B5C000EDB
:104E20000C58000E0D58000E0E5810E3A6EC4BF077
:104E300004C087FD05C088FD06C089FD07C08AFD46
:104E40000201150E216F18EC1EF089749EAAC8D7B6
:104E50000D01045101E07ED0B7EC4BF09EAA10D0BA
:104E60008974AECF01FD0D010051030A28E0010A4B
:104E700023E0030A1BE0010504E1010E006F15D0D9
:104E8000E7D7040E015D0CE1898417EC41F00201C3
:104E9000060E216F18EC1EF00D01010E046F05D0F7
:104EA0000201150E216F18EC1EF053D0060E066F8E
:104EB000056B020E006F4DD0030E006F4AD00551F6
:104EC000052BEA6A070FE96E0D0EEA2201CDEFFF0E
:104ED00005510B6E0C6A0C50000AE8AE02D00C347F
:104EE00005D0800ED8800B54000E0C5431E202CD58
:104EF000ECF303CDEDF364EC41F00D01060E066F0B
:104F0000016B01510B6E0C6A0C50000AE8AE02D026
:104F1000D89004D0800E0B5C000E0C580DE20151AD
:104F2000EA6A070FE96E0D0EEA22EFCFEEF37DEC91
:104F300041F00D01012BE5D79AEC41F0F3CF02FDD2
:104F4000F4CF03FD06CD21F218EC1EF00D01006B2D
:104F500000D07ED7010E00D01200640EE66EC4ECC5
:104F60004BF0E5521200320EE66EC4EC4BF0E55207
:104F70001200F29E050EE66EE2EC4BF0E552F28E68
:024F800012001D
:0E4F82000D01036B020E035D26E2500E0101CD
:104F90009E6F9F6BEBEC00F0E66E0D0103510A0D66
:104FA000F3CFE9FFF4CFEAFF720EE926030EEA22FF
:104FB000E552E750EF6E03510A0DF3CFE9FFF4CF4E
:104FC000EAFF720EE926030EEA22030EE926000E1E
:104FD000EA22EF6A032BD7D712000D019A6B020E5B
:104FE0009A5D06E29ACD86F304D80D019A2BF7D785
:104FF0001200030186510A0DF3CF61FDF4CF62FD6B
:10500000720E0D016127030E6223010E546F0D0114
:10501000545101E14DD2546B61CDE9FF62CDEAFFFD
:10502000EF500101A46F37EC02F000090AE161CDF5
:10503000E9FF62CDEAFF030EE926000EEA22EF6ADD
:1050400037D261CDE9FF62CDEAFF030EEB50090ACA
:1050500001E103D2080A01E1D8D10A0A01E12ED107
:10506000090A01E1E0D0020A01E021D261CDE9FFA5
:1050700062CDEAFFEF500101B36F03EC05F00009C8
:1050800001E1D0D00D01010E546F526B536B0D0135
:10509000500E525D000E535918E252CDB1F153CD6E
:1050A000B2F1522B000E5323000E0101B1270D0E59
:1050B000B22361CDE9FF62CDEAFFEF500101B06F8D
:1050C000A5EC04F0000901E0E2D7000E0D01522525
:1050D000E96E0D0E5321EA6EEF6A61CDE9FF62CDF4
:1050E000EAFFEF500101AA6F30EC04F061CDE9FF57
:1050F00062CDEAFF030EE926000EEA22020EEF6EF1
:105100000D01050E5F6F61CDE9FF62CDEAFF090E6B
:10511000E926000EEA22E9CF8FF3EACF90F30301EC
:105120005F0E8D6F0D0E8E6F0301550E8B6F0D0E82
:105130008C6F0301000E896F0D0E8A6FDBDA0D0193
:10514000516F51516FE15F51010813E25FCD39F2A8
:105150000201550E376F0D0E386FF9EC1FF061CD5F
:10516000E9FF62CDEAFF090EE926000EEA22030EEE
:10517000EF6E55CDE8F356CDE9F38CEC40F0F3CF6C
:105180000BF0F4CF0CF061CDE9FF62CDEAFF010E28
:105190000BC0EBFF020E0CC0EBFF61CDE9FF62CD4F
:1051A000EAFFEE52FF0EEE1802E1FF0EED1814E1D9
:1051B00061CDE9FF62CDEAFF080EE926000EEA2282
:1051C000EF6A61CDE9FF62CDEAFF030EE926000E2A
:1051D000EA22020EEF6E26D061CDE9FF62CDEAFF32
:1051E000EE52EE50ED1014E161CDE9FF62CDEAFF21
:1051F000080EE926000EEA22030EEF6E61CDE9FFEC
:1052000062CDEAFFE926000EEA22020EEF6E0AD016
:1052100061CDE9FF62CDEAFF030EE926000EEA2226
:105220000B0EEF6E44D161CDE9FF62CDEAFFEF5086
:105230000101A76F92EC03F000093FE061CDE9FFA7
:1052400062CDEAFF080EEB50E96EEA6AD890E936C3
:10525000EA361D0EE926040EEA22EECF63FDEDCFFD
:1052600064FD0D0163CDF6FF64CDF7FF632B000EE7
:1052700064230800F5CF60FDF5500CE060CDA9F186
:1052800061CDE9FF62CDEAFFEF500101A86FBCECF0
:1052900003F0E7D761CDE9FF62CDEAFFEF500101EE
:1052A000A66FC6EC02F061CDE9FF62CDEAFF030E06
:1052B000E926000EEA22090EEF6EF9D061CDE9FF72
:1052C00062CDEAFFEF500101A76F92EC03F00009F5
:1052D00001E19AD00D01010E546F606B60510B6EAD
:1052E0000C6A1F0E0B5C000E0C5815E26051F76A39
:1052F000680FF66E960EF7220800F5CFA9F161CD82
:10530000E9FF62CDEAFFEF500101A86FBCEC03F0AA
:105310000D01602BE3D761CDE9FF62CDEAFF090EF5
:10532000EB50140DF3CFF6FFF4CFF7FFDC0EF626AB
:10533000950EF722F6CF63FDF7CF64FD0D0163CD27
:10534000F6FF64CDF7FF632B000E64230800F5CF52
:1053500060FDF5500CE060CDA9F161CDE9FF62CDB3
:10536000EAFFEF500101A86FBCEC03F0E7D7606BD8
:1053700060510B6E0C6A040E0B5C000E0C5815E2AB
:105380006051F76A880FF66E960EF7220800F5CF87
:10539000A9F161CDE9FF62CDEAFFEF500101A86FED
:1053A000BCEC03F00D01602BE3D761CDE9FF62CDCA
:1053B000EAFF090EEB5003080BE161CDE9FF62CD76
:1053C000EAFF070EE926000EEA22010EEF6E09D071
:1053D00061CDE9FF62CDEAFF070EE926000EEA2261
:1053E000EF6A61CDE9FF62CDEAFF040EE926000E07
:1053F000EA22030EEF6E61CDE9FF62CDEAFFE926F6
:10540000000EEA22010EEF6E52D061CDE9FF62CDAF
:10541000EAFFEF500101B36F03EC05F0000909E06A
:1054200061CDE9FF62CDEAFFEF500101AA6F30ECD8
:1054300004F061CD87F362CD88F33BD800090CE01E
:1054400017EC41F061CDE9FF62CDEAFF030EE926DA
:10545000000EEA22090EEF6E2AD061CDE9FF62CD7F
:10546000EAFFEF500101A46F37EC02F000091EE0E3
:1054700061CDE9FF62CDEAFFEF500101A76F92EC29
:1054800003F0000913E061CDE9FF62CDEAFFEF50C0
:105490000101A56F4AEC02F061CDE9FF62CDEAFFA0
:1054A000030EE926000EEA220A0EEF6E00D0AFD5F9
:1054B000120087C3E9FF88C3EAFFEE52EECFEAF39A
:1054C000EDCFEBF31EEC41F087C3E9FF88C3EAFFA1
:1054D000EF500101A76F92EC03F0000901E1F7D052
:1054E0000D01986B87C3E9FF88C3EAFF040EEB50F8
:1054F000080816E032EC41F00D01996F0301E31D3D
:1055000001E1E41D0DE151EC41F087C3E9FF88C3DF
:10551000EAFFEF500101A66FC6EC02F0010EE9D0E0
:1055200087C3E9FF88C3EAFF070EEB50000901E1DA
:10553000C2D087C3E9FF88C3EAFF040EEB50080A14
:1055400066E00E0A43E0030A15E0060A01E0A4D073
:10555000250E0D01995D0BE187C3E9FF88C3EAFFC2
:10556000040EE926000EEA22050EEF6E02D0010EAF
:10557000986F93D0250E0D01995D0DE1010E986F86
:1055800087C3E9FF88C3EAFF040EE926000EEA227A
:10559000030EEF6E1AD0300E995D100DF350E66ECB
:1055A00087C3E9FF88C3EAFF080EE926000EEA2256
:1055B000E552E750EF6E87C3E9FF88C3EAFF040EA8
:1055C000E926000EEA22060EEF6E67D0300E0D01BE
:1055D000995D0B6E87C3E9FF88C3EAFF080EE926D1
:1055E000000EEA220B50EF1287C3E9FF88C3EAFFDF
:1055F000040EE926000EEA22080EEF6E87C3E9FFCB
:1056000088C3EAFF050EEB6A060EEB6A46D002017C
:10561000990E3D6F0D0E3E6F87C3E9FF88C3EAFF09
:10562000050EE926000EEA22EECF3BF2EDCF3CF26A
:1056300087C3E9FF88C3EAFF080EEB5002013A6F07
:105640005FEC20F0F3CF0BF0F4CF0CF087C3E9FF51
:1056500088C3EAFF050E0BC0EBFF060E0CC0EBFF84
:105660000D01010E986F87C3E9FF88C3EAFF050E9D
:10567000E926000EEA22FF0EEE1802E1FF0EED18F9
:105680000AE187C3E9FF88C3EAFF040EE926000E9A
:10569000EA22030EEF6E01D0FFD798510BE099CDAF
:1056A000A9F187C3E9FF88C3EAFFEF500101A86FA2
:1056B000BCEC03F00BD099CDA9F187C3E9FF88C3F7
:1056C000EAFFEF500101A86FBCEC03F0FDD651ECEE
:1056D00041F0F3CF0BF0F4CF0CF087C3E9FF88C3A0
:1056E000EAFF010E0BC0EBFF020E0CC0EBFF000E39
:1056F00000D012000D01666B686B696B656B030E61
:10570000E66EE66A8D0E0B6E960E0C6E0D6A0BC081
:10571000E6FF0CC0E6FF0DC0E6FF89C3E6FF8AC3C3
:10572000E6FF64EC47F0F56E070EE15EF550000908
:1057300008E1040E03018927000E8A230D01676B1F
:1057400002D0020E4AD189C3E9FF8AC3EAFFEF50B3
:10575000200805E10301892B000E8A23F4D789C3B1
:10576000E9FF8AC3EAFFEFCF6AFD200E0D016A5DF3
:1057700001E1A7D06A5101E1A4D00D0E6A5D01E1FB
:10578000A0D00A0E6A5D01E19CD08DC3E9FF8EC3F3
:10579000EAFFEF50655D01E394D06651020A33E001
:1057A000030A20E0010A01E081D06551020D0301E6
:1057B0008B51F324E96E8C51F420EA6E89C3EEFF1D
:1057C0008AC3EDFF89C3E9FF8AC3EAFFEFCF6AFD11
:1057D0002F0E0D016A5D03E05C0E6A5D02E1010EB1
:1057E000666F64D06551652B020D03018B51F32464
:1057F000E96E8C51F420EA6E89C3EEFF8AC3EDFF97
:105800000D01020E666F89C3E9FF8AC3EAFFEFCF7D
:105810006AFD3F0E6A5D03E0260E6A5D08E189C3FA
:10582000E9FF8AC3EAFFEF6A010E666F3ED02B0ED6
:105830006A5D07E1200E89C3E9FF8AC3EAFFEF6EC4
:1058400034D02E0E6A5D0BE1650509E10301892B59
:10585000000E8A2389C368FD8AC369FD26D03D0EE8
:105860006A5D08E189C3E9FF8AC3EAFFEF6A010EB6
:10587000666F1BD02F0E6A5D03E05C0E6A5D15E15A
:10588000010E03010C6A89250B6E8A510C220D0151
:105890006505020D03018B51F324E96E8C51F42050
:1058A000EA6E0BC0EEFF0CC0EDFF00D00301892BA8
:1058B000000E8A2389C3E9FF8AC3EAFFEFCF6AFD9E
:1058C00054D789C3E9FF8AC3EAFFEF6A070E8FC383
:1058D000E9FF90C3EAFFEF6E6851691142E068CDBD
:1058E000E6FF69CDE6FF59EC48F0E552E552F3CF0B
:1058F00068FDF4CF69FD0D01C00E6B6F950E6C6FE6
:105900006A6B6A510B6E0C6A070E0B5C000E0C582A
:1059100028E2030EE66EE66A6BCD0BF06CCD0CF060
:105920000D6A0BC0E6FF0CC0E6FF0DC0E6FF68CDB8
:10593000E6FF69CDE6FF64EC47F0F56E070EE15E29
:10594000F550000907E18FC3E9FF90C3EAFF6ACD74
:10595000EFFF07D0040E0D016B27000E6C236A2B9E
:10596000D0D70D01655131E1090EE66EE66A910E60
:105970000B6E960E0C6E0D6A0BC0E6FF0CC0E6FFB8
:105980000DC0E6FF8BC3E9FF8CC3EAFFEECFE6FF55
:10599000EFCFE6FFAEEC47F0F56E070EE15EF55097
:1059A0008BC3E9FF8CC3EAFFEE50EFCFEAFFE96E4D
:1059B000090EE926000EEA22EF6A010E8FC3E9FF05
:1059C00090C3EAFFEF6E0D01652B8DC3E9FF8EC317
:0C59D000EAFF65CDEFFF675100D0120028
:0459DC000001D38172
:1059E000F5DA0A0EE66EC4EC4BF0E5520001ED6B01
:1059F00000010E0EEC6FFADA0001800EED6F00016F
:105A0000050EEC6FF3DA0001020EED6F00010E0ED1
:105A1000EC6FECDA0001400EED6F0001EC6BE6DAA2
:105A20000001EE6BEDDA0D01036F03B1F9D7000150
:105A3000ED6B00010D0EEC6FD9DA0001010EED6F78
:105A400000010E0EEC6FD2DA00010C0EEE6FD8DA08
:105A50000D01036F03B3F8D70001ED6B00010D0ECC
:105A6000EC6FC4DA0001040EED6F00010C0EEC6F58
:105A7000BDDA08C2EDF00001040EEC6FB7DA09C21E
:105A8000EDF00001050EEC6FB1DA0AC2EDF0000195
:105A9000060EEC6FABDA0BC2EDF00001070EEC6FF7
:105AA000A5DA0CC2EDF00001080EEC6F9FDA0DC212
:105AB000EDF00001090EEC6F99DA0001ED6B0001C9
:105AC0000E0EEC6F93DA0001810EED6F0001EC6BAE
:105AD0008DDA0001040EED6F0001EC6F87DA000132
:105AE000010EED6F0001050EEC6F80DA0001100E63
:105AF000ED6F00010A0EEC6F79DA0001080EED6F10
:105B000000010B0EEC6F72DA0001F76B800EF86F7C
:105B10000001020EF66F12DB0001020EF56FEBDAE8
:105B2000F3CF04FDF4CF05FD05CD03FD0D0103BF4B
:105B3000F3D70001E10EF76F010EF86F0001120EAE
:105B4000F66FFCDA0001F76B320EF86F0001020EFF
:105B5000F66FF4DA0001020EED6F00010E0EEC6F2D
:105B600045DA58EF2EF00001ED6B00010E0EEC6FE0
:105B70003DDA0001020EEE6F43DA0D018B6F00017A
:105B8000020EED6F00010E0EEC6F30DA0001D35102
:105B9000010B06E10D018B51010B02E1000E01D05A
:105BA000010E00D01200010E00D012000001060EFE
:105BB000EE6F26DA0D01DA6F0001070EEE6F20DAC4
:105BC0000D01D96FD99BDACDEDF00001060EEC6F17
:105BD0000DDAD9CDEDF00001070EEC6F07DAD8C071
:105BE000EDF00001080EEC6FF6EF2FF00001DBC0C6
:105BF0000BF0DCC00CF0DB07000EDC5B0B500C1074
:105C00000EE0D9C0E9FFDAC0EAFFD92B000EDA2393
:105C1000EFCFEDF00001080EEC6FE8D9E7D71200E6
:105C20000001060EEE6FECD90D01B26F0001070EF8
:105C3000EE6FE6D90D01B16FB18BB2CDEDF0000181
:105C4000060EEC6FD3D9B1CDEDF00001070EEC6F6D
:105C5000CDD90001080EEE6FD3D900D01200DFC0FD
:105C600031FDE0C032FD0001DFC00BF0E0C00CF000
:105C7000DF07000EE05B0B500C1011E00001080E76
:105C8000EE6FBED9E66E0001DDC0E9FFDEC0EAFFBF
:105C9000DD2B000EDE23E552E750EF6EE4D731CD69
:105CA000F3FF32CDF4FF00D012000001D3911200B7
:105CB0000001240EED6F0001EC6B98D900010C0E71
:105CC000EE6F9ED90D01006F00A7F8D70001030EFB
:105CD000EE6F96D90D01006F00AF02D0FF0E18D005
:105CE00000CDD7F0D7C0EDF00001020EEC6F7ED9E9
:105CF0000001ED6B0001060EEC6F78D90001400E3B
:105D0000ED6F0001070EEC6F71D90001D75100D083
:105D100012000001D38112000001ED6B00010C0E96
:105D2000EC6F64D90001800EED6F0001EC6B5ED961
:105D30000001EE6B65D90D01B16FB1B1F9D7120059
:105D40000001ED6B00010E0EEC6F50D90D018B6B55
:105D50000001090EEE6F54D90D018C6F080E8C03F3
:105D6000F3CF8CFD0001020EED6F00010E0EEC6F03
:105D70003DD98BCD8DFD8CCD8EFD8BCDF3FF8CCDA4
:105D8000F4FF00D01200E5C0E9FFE6C0EAFFEF68CB
:105D90000001050EEE6F34D90D010E6F0EAF02D06B
:105DA000000E6DD00ECDD6F00001ED6B0001060E99
:105DB000EC6F1CD90001E00EED6F0001070EEC6FD7
:105DC00015D90001080EEE6F1BD90D01106F0001EF
:105DD000080EEE6F15D90D010E6F0001080EEE6F63
:105DE0000FD90D01116F0001080EEE6F09D90D01D9
:105DF000126F0ECD0FFDA80E0E1503E08DDF000E05
:105E00003ED00E0E0001DF6FE06B0001000EDD6F73
:105E10000D0EDE6F24DF0CCD0AF40DCD0BF46EEC0D
:105E200048F0F3CF0CFDF4CF0DFD060EE66EE66AEA
:105E3000060EE66E0D0EE66EE3C0E9FFE4C0EAFF73
:105E4000E9CF0BF0EACF0CF00BC0E6FF0CC0E6FF89
:105E500083EC47F0F56E060EE15EF550080E0D017D
:105E60000D5D0BE10C5103E0060E0C5D06E1E5C093
:105E7000E9FFE6C0EAFF0CCDEFFF010E00D01200F3
:105E80000E0E0001EA25D46F000EEB21D56F000144
:105E9000ED6B0001060EEC6FA9D80001400EED6F0E
:105EA0000001070EEC6FA2D80001ED6B0001080E97
:105EB000EC6F9CD80001ED6B0001080EEC6F96D8DA
:105EC000D4C0D3FDD5C0D4FD060E0D01D327000EDE
:105ED000D423D3CDD6FDD4CDD7FDD3CDEDF0000165
:105EE000080EEC6F83D8D4CDEDF00001080EEC6FF6
:105EF0007DD8060E0001DB6FDC6BE7C0D9F0E8C08F
:105F0000DAF074DE08C2D8F051DE09C2D8F04EDEF5
:105F10000AC2D8F04BDE0BC2D8F048DE0CC2D8F073
:105F200045DE0DC2D8F042DE0001E95103E10D016A
:105F3000D86B03D00D01060ED86F0001080ED86F84
:105F400035DED8CDD8F0D6EF2DF0040E0001D427E1
:105F5000000ED523D4C0EDF00001060EEC6F46D83C
:105F6000400E0001D5110001ED6F0001070EEC6F2E
:105F70003DD80001D4A108D00001200EED6F000132
:105F8000080EEC6F33D80CD00001ED6B0001080E49
:105F9000EC6F2CD80001ED6B0001080EEC6F26D8D9
:105FA000D7C0EDF00001020EEC6F20D80001C00E4A
:105FB000ED6F0001EC6B1AD80001ED6B0001010ED2
:105FC000EC6F14D80001D3A1D381120095680001B1
:105FD000F46B83D8F19E848284808484966A050E53
:105FE000E66EE2EC4BF0E55284941200ECC0F4F063
:105FF00074D8EDC083FF956A8492848295681200FC
:106000009568EEC0F4F069D8849083CFDCFD84807D
:106010000D01DC5100D012000D01B26B120EB16FF8
:106020000001EF510D01B1270001F0510D01B22324
:10603000030EB115B36FFC0EB117B1CDEDF0000139
:10604000060EEC6FD3DFE00E0D01B2110001ED6F13
:106050000001070EEC6FCADF0D01B351B307000951
:1060600005E00001080EEE6FCBDFF6D71200F1C09D
:10607000EDF00001020EEC6FB9DF0D01B26B120EF4
:10608000B16F0001F2510D01B1270001F3510D0173
:10609000B223B1CDEDF00001060EEC6FA7DF400E8C
:1060A0000D01B2110001ED6F0001070EEC6FF6EF6C
:1060B0002FF00001070EEE6FA3DF0D01016F070E39
:1060C00001170001060EEE6F9BDF0D01006F00CD82
:1060D000F3FF01CDF4FF00D01200F4C0DBFD0D0191
:1060E000DB51010B02E0DB9901D0DB89DBCD81FFC5
:1060F000E00E936E1200F5C0FAF00001600EF96F29
:106100003AD8F5C0FBF083D80D01076FF5C0FBF05E
:106110007ED80D01066F0001ED6B0001080EEC6FDB
:1061200065DF0001040EED6F0001080EEC6F5EDF0D
:1061300006CDF3FF07CDF4FF00D01200F6C0FAF051
:106140000001500EF96F17D8F7C000FDF8C001FD2F
:106150000001080EFD6F01CDFCF088D80001080E8B
:10616000FD6F00CDFCF082D80001ED6B0001080E40
:10617000EC6FF6EF2FF00001030EED6F00010E0E35
:10618000EC6F34DF0D01026B200E025D16E20001A0
:10619000090EED6F0001080EEC6F28DF050EE66EAC
:1061A000C4EC4BF0E55200010D0EED6F0001080E3E
:1061B000EC6F1CDF0D01022BE7D7050EE66EC4EC79
:1061C0004BF0E5520001080EFD6FF9C0FCF04ED80F
:1061D000600E0001F95D14E10001060EFD6FFAC0CA
:1061E000FCF044D80001ED6B0001080EEC6FFEDE00
:1061F0000001040EED6F0001080EEC6FF7DE06D013
:106200000001080EFD6FFAC0FCF030D812000D013D
:10621000026B080E025D27E20001080EEE6FF0DE51
:106220000D01006F00A302D0018101D00191000196
:10623000ED6B0001080EEC6FD9DE050EE66EC4ECC6
:106240004BF0E5520001040EED6F0001080EEC6FFB
:10625000CDDE050EE66EC4EC4BF0E5520D01019F5C
:106260000147022BD6D7015100D01200FCC008FD17
:106270000D01096B0001FD510D01095D32E208AF0E
:1062800014D00001090EED6F0001080EEC6FAEDEB8
:10629000050EE66EC4EC4BF0E55200010D0EED6FFD
:1062A0000001080EEC6FA2DE12D00001080EED6FA7
:1062B0000001EC6F9BDE050EE66EC4EC4BF0E55280
:1062C00000010C0EED6F0001080EEC6F8FDE050E65
:1062D000E66EC4EC4BF0E5520D01089F0847092B10
:0462E000C9D7120008
:0C62E400070E0201FB5D01E10BD0FF0E74
:1062F000FC5D04E0FCC233F323EC36F00201FC69E0
:10630000FB6BFE6B12000201FB51060A01E11BD17F
:10631000030A01E1BAD0010A01E19FD0070A73E044
:10632000010A4FE0030A31E0010A01E03AD10D0110
:1063300000690169026903690469056906690769F9
:10634000086909690301996B9A6B9B6B9C6B430EFF
:106350000301316F326B0301000E2F6F0D0E306F92
:10636000440E03012D6F2E6BB8EC35F00201FC6F6B
:10637000A6EC4BF004C0A5F305C0A6F306C0A7F336
:1063800007C0A8F30201010EFB6FA6EC4BF003015E
:10639000A551045C0B6EA65105580C6EA75106580A
:1063A0000D6EA85107580E6E140E0B5C000E0C58A3
:1063B000000E0D58000E0E5803E30201020EFB6F93
:1063C000F0D0030199519A119B119C1104E0020134
:1063D000040EFB6F17D0FCC22CF3B3EC2DF00009B8
:1063E00011E00301010EA96F9DDAA6EC4BF004C089
:1063F000A5F305C0A6F306C0A7F307C0A8F30201E2
:10640000030EFB6FCED0A6EC4BF00301A551045C4C
:106410000B6EA65105580C6EA75106580D6EA8516B
:1064200007580E6EC80E0B5C000E0C58000E0D586F
:10643000000E0E5803E30201020EFB6FFCC235F39F
:1064400037EC37F0000908E0B4D8020804E1020193
:10645000040EFB6F02D0A5D0A4D0FCC22CF3B3EC89
:106460002DF0000911E00301030EA96F5BDAA6EC21
:106470004BF004C0A5F305C0A6F306C0A7F307C000
:10648000A8F30201050EFB6F8CD0FCC235F337EC8C
:1064900037F000093CE08DD80D010A6F060E0A5D49
:1064A00004E10201040EFB6F31D0050E0A5D2EE1FE
:1064B000FCC233F323EC36F00201FC69A6EC4BF08E
:1064C00004C0A5F305C0A6F306C0A7F307C0A8F350
:1064D0000201060EFB6F99C304F29AC305F29BC337
:1064E00006F29CC307F2A1C30EF2A2C30FF2A3C32C
:1064F00010F2A4C311F29DC312F29EC313F29FC304
:1065000014F2A0C315F2FD81FE2B4BD01BD0A6ECDC
:106510004BF00301A551045C0B6EA65105580C6E9F
:10652000A75106580D6EA85107580E6EC80E0B5C89
:10653000000E0C58000E0D58000E0E5803E3020119
:10654000020EFB6F2ED0A6EC4BF00301A551045CAC
:106550000B6EA65105580C6EA75106580D6EA8512A
:1065600007580E6E640E0B5C000E0C58000E0D5892
:10657000000E0E5816E39507000E965B975B985B2E
:10658000955196119711981102E10201FB6BA6EC4F
:106590004BF004C0A5F305C0A6F306C0A7F307C0DF
:1065A000A8F312000201080EFB6FFCC233F323EFC5
:1065B00036F00D010D6B03013C0E956F966B976BDA
:1065C000986B03010B0E366F0D0E376F52EC37F0E0
:1065D000020E0D010B5D01E07DD10C6B0F0E0C5D09
:1065E0000AE203010B0E366F0D0E376F52EC37F0D7
:1065F0000D010C2BF3D70301990E366F030E376F85
:1066000052EC37F003019A0E366F030E376F52ECDF
:1066100037F003019B0E366F030E376F52EC37F0E5
:1066200003019C0E366F030E376F52EC37F00D01ED
:106630000C6B080E0C5D0AE203010B0E366F0D0E9B
:10664000376F52EC37F00D010C2BF3D70C6B060EA5
:106650000C5D14E203010B0E366F0D0E376F52EC1A
:1066600037F00D010C51EA6A080FE96E020EEA22BA
:10667000EF500B5D01E051D10C2BE9D70C6B0C51A5
:106680000B6E0C6A0C50000AE8AE02D0D89004D011
:10669000CE0E0B5C000E0C580AE203010B0E366F97
:1066A0000D0E376F52EC37F00D010C2BE8D70E6B47
:1066B00003010B0E366F0D0E376F52EC37F00D01E4
:1066C0000B51330A01E1B2D0CC0A01E1ACD0C90AC6
:1066D00001E17FD0350A43E0020A17E0340A01E005
:1066E000E1D003010B0E366F0D0E376F52EC37F011
:1066F0000D010B0508E103010D0E366F0D0E376F0E
:1067000052EC37F001D009D1E1D003010B0E366F06
:106710000D0E376F52EC37F0040E0D010B5D1DE1CD
:106720000301A10E366F030E376F52EC37F00301F1
:10673000A20E366F030E376F52EC37F00301A30E33
:10674000366F030E376F52EC37F00301A40E366F2D
:10675000030E376F52EC37F001D0DFD0B7D0030112
:106760000B0E366F0D0E376F52EC37F0040E0D0125
:106770000B5D1DE303019D0E366F030E376F52EC68
:1067800037F003019E0E366F030E376F52EC37F071
:1067900003019F0E366F030E376F52EC37F0030183
:1067A000A00E366F030E376F52EC37F001D0B5D024
:1067B000040E0D010B5F0D010B510B07000908E0E2
:1067C00003010C0E366F0D0E376F52EC37F0F3D716
:1067D0007DD003010B0E366F0D0E376F52EC37F084
:1067E000040E0D010B5D1DE10301120E366F0D0E3F
:1067F000376F52EC37F00301110E366F0D0E376F05
:1068000052EC37F00301100E366F0D0E376F52EC5D
:1068100037F003010F0E366F0D0E376F52EC37F065
:1068200001D07BD053D0010E0E6F50D003010B0E60
:10683000366F0D0E376F52EC37F0040E0D010B5D05
:106840002FE10301980E366F030E376F52EC37F0CD
:106850000301970E366F030E376F52EC37F00301CA
:10686000960E366F030E376F52EC37F00301950E1C
:10687000366F030E376F52EC37F0080ED8800301E5
:106880009555070E9655000E9755000E985507E240
:10689000080E955F070E965B000E975B985B01D024
:1068A0003CD014D003010B0E366F0D0E376F52EC37
:1068B00037F00D010B510B07000908E003010C0E26
:1068C000366F0D0E376F52EC37F0F3D70D010E51C6
:1068D00001E1EED6020E0D5D09E10FCD91F310CD71
:1068E00092F311CD93F312CD94F312D0910EE96E81
:1068F000030EEA6EEE500F1909E1EE50101906E191
:10690000EE50111903E1EE50121900E101E00D6B98
:10691000BAEC37F00D010D5104D0BAEC37F0000E8F
:1069200000D012000301010E346F35EC36F0030184
:10693000010E346F35EC36F00301060E346F35EC82
:1069400036F00301346B35EC36F00301120E346F70
:1069500035EC36F00301230E346F35EC36F00301CD
:10696000340E346F35EC36F00301560E346F35ECCF
:1069700036F00301346B35EC36F00301346B35EC43
:1069800036F00301800E346F35EC36F00301346BC2
:1069900035EC36F00301346B35EC36F00301346B23
:1069A00035EC36F00301346B35EC36F00301346B13
:1069B00035EC36F00D010B6B0C0E0B5D07E203019D
:1069C000346B35EC36F00D010B2BF6D708C234F3DF
:1069D00035EC36F009C234F335EC36F00AC234F344
:1069E00035EC36F00BC234F335EC36F00CC234F330
:1069F00035EC36F00DC234F335EC36F00D010B6B8F
:106A00000B510B6E0C6A0C50000AE8AE02D0D89005
:106A100004D0CA0E0B5C000E0C5807E20301346B65
:106A200035EC36F00D010B2BEBD70301630E346F01
:106A300035EC36F00301820E346F35EC36F003018D
:106A4000530E346F35EC36F00301630E346F35ECC2
:106A500036F00301350E346F35EC36F00301010ECC
:106A6000346F35EC36F0A9C334F335EC36F003015E
:106A7000A9051FE099519A119B119C111AE003017D
:106A8000360E346F35EC36F00301040E346F35ECFE
:106A900036F094C334F335EC36F093C334F335EC6D
:106AA00036F092C334F335EC36F091C334F335EC61
:106AB00036F00301370E346F35EC36F00301020E69
:106AC000346F35EC36F00301010E346F35EC36F0DF
:106AD0000301030E346F35EC36F0030E0301A95D9C
:106AE0001AE10301320E346F35EC36F00301040E67
:106AF000346F35EC36F099C334F335EC36F09AC385
:106B000034F335EC36F09BC334F335EC36F09CC3EC
:106B100034F335EC36F00301346935EC36F0ACEF84
:026B200036F04D
:0E6B22000D01006B020E005D21E20051160D08
:106B3000F3CFE9FFF4CFEAFF000EE926030EEA22C5
:106B40000C0EE926000EEA22EE6AED6A0051160DDF
:106B5000F3CFE9FFF4CFEAFF000EE926030EEA22A5
:106B6000150EE926000EEA22EF90002BDCD712006A
:106B70000D01000E0C6F030E0D6F0B6B020E0B5D03
:106B80005FE20CCDE9FF0DCDEAFF0C0EE926000E09
:106B9000EA22EECF0BF0EFCF0CF00D6A0E6A0B502D
:106BA0000C100D100E1046E10CCDE9FF0DCDEAFFE3
:106BB0000C0E2DC3EBFF0D0E2EC3EBFF03012F5167
:106BC000301119E00A0EE66EE66A2FC3E6FF30C305
:106BD000E6FF0CCDE9FF0DCDEAFFE9CF0BF0EACFE0
:106BE0000CF00BC0E6FF0CC0E6FF83EC47F0F56E3F
:106BF000060EE15EF5500CCDE9FF0DCDEAFF0A0E61
:106C000031C3EBFF0B0E32C3EBFF0CCDE9FF0DCD13
:106C1000EAFF0E0EEB6A0F0EEB6A0CCDE9FF0DCD0D
:106C2000EAFF100EEB6A110EEB6A0BCD2CF30D018F
:106C30000B5108D0160E0C27000E0D230B2B9ED7E0
:106C4000FF0E00D0120003013351160DF3CFE9FF00
:106C5000F4CFEAFF000EE926030EEA220C0EE92625
:106C6000000EEA22EE6AED6A120003012C51160DA5
:106C7000F3CFE9FDF4CFEAFD000E0D01E927030E85
:106C8000EA23E9CDE9FFEACDEAFF0E0EE926000E80
:106C9000EA22EE50ED101DE1E9CDE9FFEACDEAFF71
:106CA000120ED7C0EBFF1C0E0001F26FF36BE9CDA3
:106CB000E9FFEACDEAFF120EEB500001F16F37EC6D
:106CC00030F0E9CDE9FFEACDEAFF130EEB6A140ECE
:106CD000EB6A34C3D8F0D6EC2DF0E9CDE9FFEACD6C
:106CE000EAFF130EE926000EEA22EECF0BF0EDCFFD
:106CF0000CF0EE2AEF22E9CDE9FFEACDEAFF0E0E15
:106D0000E926000EEA22EECF0DF0EFCF0EF00D5087
:106D10000B5C0E500C580AE3E9CDE9FFEACDEAFF1F
:106D20000E0EE926000EEA22EE2AEF22E9CDE9FF57
:106D3000EACDEAFF0E0EE926000EEA22EECFEBFDC9
:106D4000EDCFECFD0D01D60EEB5D030EEC5901E32A
:106D500003D8010E00D0120003012C51160DF3CF01
:106D6000E7FDF4CFE8FD000E0D01E727030EE82351
:106D7000E7CDE9FFE8CDEAFF0C0EE926000EEA2296
:106D8000EECF0AF4EDCF0BF46EEC48F0F3CFDFFD5D
:106D9000F4CFE0FDE7CDE9FFE8CDEAFF0A0EE926F2
:106DA000000EEA22EECF0AF4EDCF0BF46EEC48F0C1
:106DB000F3CFE1FDF4CFE2FDE7CDE9FFE8CDEAFF57
:106DC0000E0EE926000EEA22EECFE3FDEFCFE4FD42
:106DD000080E0D01E327000EE423E56BE66B140EAD
:106DE0000001F26FF36BE7CDE9FFE8CDEAFF120E89
:106DF000EB500001F16F37EC30F0E3CDFCF3E4CD64
:106E0000FDF30301110EFB6FE7CDE9FFE8CDEAFFCB
:106E1000E9CFF9F3EACFFAF34AEC3EF0E3CD0AF416
:106E2000E4CD0BF46EEC48F0F3CFE3FDF4CFE4FDDA
:106E3000080E0001DB6FDC6B0001DF0ED96F0D0E59
:106E4000DA6FF6EC2DF0A5EC2FF0E7CDE9FFE8CDF9
:106E5000EAFF120EE926000EEA22EF68E7CDE9FF0D
:106E6000E8CDEAFF0E0EEB6A0F0EEB6A120035C397
:106E70002CF303012C51160DF3CFE9FFF4CFEAFFF9
:106E8000000EE926030EEA22100EE926000EEA2281
:106E9000D880EE54000EED5402E3000E01D0010E36
:106EA00000D0120003012C51160DF3CFE9FFF4CFEF
:106EB000EAFF000EE926030EEA22100EE926000E74
:106EC000EA22EE50ED1002E1000E53D02C51160DC7
:106ED000F3CFE9FFF4CFEAFF000EE926030EEA2222
:106EE000150EE926000EEA22EF50010B15E02C5199
:106EF000160DF3CFE9FFF4CFEAFF000EE926030EEB
:106F0000EA22150EE926000EEA22EF901C0E00017F
:106F1000EF6FF06B0CEC30F010EC2EF036C3E9FFA5
:106F200037C3EAFFEF6E03012C51160DF3CFE9FFD3
:106F3000F4CFEAFF000EE926030EEA22100EE9263E
:106F4000000EEA22EE06EF5A2C51160DF3CFE9FFA0
:106F5000F4CFEAFF000EE926030EEA22100EE9261E
:106F6000000EEA22EE50ED1002E18CEC2EF0010E44
:106F700000D0120003012C51160DF3CFE9FFF4CF1E
:106F8000EAFF000EE926030EEA22100EE926000EA3
:106F9000EA22EE50ED1002E08CEC2EF003012C51B1
:106FA000160DF3CFE9FFF4CFEAFF000EE926030E3A
:106FB000EA22100EE926000EEA22EE6AED6A1200BD
:106FC000080E0001DF6FE06B0001000EDD6F0D0E9B
:106FD000DE6F2FEC2EF000CD0AF401CD0BF46EEC39
:106FE00048F0F3CF00FDF4CF01FD02CD0AF403CD4C
:106FF0000BF46EEC48F0F3CF02FDF4CF03FD04CDAB
:107000000AF405CD0BF46EEC48F0F3CF04FDF4CF99
:1070100005FD0D01080E045F000E055B06CD0AF4A8
:1070200007CD0BF46EEC48F0F3CF06FDF4CF07FD6F
:1070300038C33EF339C33FF30301000E3C6F0D0E1E
:107040003D6F2CD80D01086FFF0E085D03E18CEC3D
:107050002EF021D00851160DF3CFE9FFF4CFEAFF4F
:10706000000EE926030EEA22100EE926000EEA229F
:1070700004CDEEFF05CDEDFF0851160DF3CFE9FF6E
:10708000F4CFEAFF000EE926030EEA22150EE926E8
:10709000000EEA22EF80010E00D012000D010A69F5
:1070A000000E0B6F030E0C6F096B020E095D01E3FE
:1070B00091D00BCDE9FF0CCDEAFF0C0EE926000EB6
:1070C000EA22EECF0BF0EFCF0CF03CC3E9FF3DC35B
:1070D000EAFF020EE926000EEA22EECF0DF0EFCF16
:1070E0000EF00D500B1802E10E500C186CE10BCD98
:1070F000E9FF0CCDEAFF0A0EE926000EEA22EECFE8
:107100000BF0EFCF0CF03CC3E9FF3DC3EAFFEECF3D
:107110000DF0EFCF0EF00D500B1802E10E500C18D1
:1071200050E10BCDE9FF0CCDEAFF100EE926000E71
:10713000EA22EECF0FF0EFCF10F0116A126A0F5073
:107140001010111012103DE13EC3E9FF3FC3EAFFEA
:10715000060EE926000EEA22EECF0BF0EECF0CF081
:10716000EECF0DF0EFCF0EF00BCDE9FF0CCDEAFF27
:10717000060EE926000EEA22EE5000010B1909E185
:10718000EE500C1906E1EE500D1903E1EE500E1908
:1071900000E114E00BCDE9FF0CCDEAFF060EE92675
:1071A000000EEA22E868EE1808E1E868EE1805E14A
:1071B000E868EE1802E1E868EE1803E10D010951F4
:1071C00044D009CD0AFD0D01160E0B27000E0C232D
:1071D000092B6BD7FF0E0A5D35E00A51160DF3CF70
:1071E0000BFDF4CF0CFD000E0B27030E0C230A0E33
:1071F000E66EE66A3EC3E6FF3FC3E6FF0BCDE9FF5E
:107200000CCDEAFFE9CF0BF0EACF0CF00BC0E6FFA4
:107210000CC0E6FF83EC47F0F56E060EE15EF5501C
:107220003CC3E9FF3DC3EAFFEECF0BF0EFCF0CF01C
:107230000BCDE9FF0CCDEAFF0A0E0BC0EBFF0B0EE6
:0C7240000CC0EBFF0D010A5100D0120041
:04724C00150E010119
:107250009E6F9F6BEBEC00F00201696F6D6B9C6B96
:10726000686B140E6B6F6C6B120069C2A4F137EC83
:1072700002F0000909E102019C6B070E6F6F6D6B54
:10728000686B6E6B010EEAD069C2B3F103EC05F0D6
:1072900000093EE0A6EC4BF004C0ACF205C0ADF234
:1072A00006C0AEF207C0AFF20101000EB16F0D0EC5
:1072B000B26F69C2B0F1A5EC04F000090FE0020161
:1072C0009C519C2BEA6A7B0FE96E020EEA2200CDEC
:1072D000EFFF1F0E9C5D01E19C6BE6D769C2AAF12E
:1072E00030EC04F00A0E0D01005D11E102019C5129
:1072F000EA6A7B0FE96E020EEA22EF6A9C6B19DAEA
:107300009DC2B3F29EC2B4F2D9D902016F6F36D0DA
:1073100002016D5133E0A6EC4BF004C001FD05C045
:1073200002FD06C003FD07C004FDAC0EE96E020EAF
:10733000EA6EEE500D01015D016FEE500259026FD1
:10734000EE500359036FEE500459046F500E015D67
:10735000460E0259000E0359000E04590FE3A6EC25
:107360004BF004C0ACF205C0ADF206C0AEF207C0EF
:10737000AFF20201020E6F6F010E6D6F02016D51CF
:10738000010A4AE0050A0EE0040A01E065D0706BCC
:10739000A6EC4BF004C0ACF205C0ADF206C0AEF2F4
:1073A00007C0AFF269C2A7F192EC03F0000901E156
:1073B000F9D769C2A7F192EC03F000092DE070C281
:1073C000E9FFEA6AE9BEEA68D890E936EA36E70EEC
:1073D000E926010EEA22EECF05FDEDCF06FD0D01F7
:1073E00005CDF6FF06CDF7FF052B000E062308009E
:1073F000F5CF00FDF55007E000CDA9F169C2A8F175
:10740000BCEC03F0ECD769C2A6F1C6EC02F00201B5
:107410000B0E706F010E6D6F070E02016F5D1BE0AA
:107420006FC2B2F21CD800090FE00B0E0201705DB2
:1074300003E0040E6D6F04D0020E6F5D01E16D6B11
:10744000070E6F6F6E6B07D00B0E0201705D03E0CD
:10745000040E6D6FA7D700D0010E00D012000201FC
:10746000B251050A5AE0060A56E0070A3CE0060A4D
:1074700038E0030A1BE0010A03E0050E706F57D0E5
:1074800068816893010E706F0A0EE66EE66A9FC20D
:10749000E6FFA0C2E6FF710EE66E020EE66E2BEC72
:1074A00048F0F56E060EE15EF55041D068B103D0AC
:1074B000060E706F15D09FC241F2A0C242F20201C7
:1074C000710E3F6F020E406FFDEC20F0000905E0E9
:1074D00002016883020E706F03D00201060E706F06
:1074E00026D028D826D0A7C2E6FFA8C2E6FF47ECE0
:1074F00045F0E552E552F3CF6CF2A9C2E6FFAAC20D
:10750000E6FF47EC45F0E552E552F3CF6BF202019E
:107510000A0E706F0CD04AD80CD00A0E706FFE0E97
:107520006A5D04E06AC2A5F14AEC02F000D0010EE7
:1075300000D0120002016E51030A24E0020A17E093
:10754000010A01E030D0020E6E5D02E117EC41F05D
:10755000FE0E02016A5D0AE017EC41F06AC2A5F175
:107560004AEC02F00201010E6E6F1DD006D06AC215
:10757000A4F137EC02F0000904E10201030E706F80
:107580006E6F11D069C2A7F192EC03F000090AE016
:1075900069C2A4F137EC02F0000904E069C2A5F168
:1075A0004AEC02F000D0000E00D0120002016E5131
:1075B000020A3BE0030A26E0010A01E07CD068B33E
:1075C00005D0060E706F010E78D01BD0070E706FBD
:1075D0006BC2A2F16CC2A3F16951260DF3CFE9FF92
:1075E000F4CFEAFF000EE926010EEA22EE52E9CFBF
:1075F000A0F1EACFA1F151EC01F002016A6F010E96
:107600006E6F59D06AC2A4F137EC02F000090CE0A9
:107610000301E25109E159EC41F0F3CFB0F2F4CFAC
:10762000B1F20201020E6E6F46D06AC2B3F103ECF2
:1076300005F000092BE0A6EC4BF004C0ACF205C04D
:10764000ADF206C0AEF207C0AFF2B0C2ECF3B1C209
:10765000EDF364EC41F001010B0EB16F0D0EB26F52
:107660006AC2B0F1A5EC04F0000905E00BCDEEF321
:107670007DEC41F0F0D79AEC41F0F3CFB0F2F4CFCB
:10768000B1F26AC2AAF130EC04F015D06AC2A4F1DA
:1076900037EC02F000090FE19AEC41F017EC41F0F1
:1076A0006AC2A5F14AEC02F00201FE0E6A6F090EF1
:1076B000706F010E02D0000E00D012000D01076B9A
:1076C000060EE76E0719E8AE02D0E73402D0E750A5
:1076D000075D2CE2040EE66EE66A07CDE9FFEA6A72
:1076E000E9BEEA68D890E936EA36DB0EE926010EF3
:1076F000EA22EECF0BF0EFCF0CF00D6A0BC0E6FFE5
:107700000CC0E6FF0DC0E6FFB3C2E6FFB4C2E6FF61
:1077100064EC47F0F56E070EE15EF550000903E1F9
:107720000D01075105D00D01072BCAD7060E00D059
:1077300012000D010A6B7B0E076F020E086F07CD5A
:10774000E9FF08CDEAFFEF50200804E1072B000E07
:107750000823F5D707CD9DF208CD9EF20201010E58
:10776000AB6F07CDE9FF08CDEAFFEFCF09FDEF5082
:107770003BE00D010A51010A1DE0010A01E030D091
:10778000200E095D03E02C0E095D08E107CDE9FF3D
:1077900008CDEAFFEF6A010E0A6F0BD00D0E095DEE
:1077A00003E00A0E095D05E107CDE9FF08CDEAFF18
:1077B000EF6A16D0200E095D12E00201AB51AB2B2F
:1077C000E96EEA6AD890E936EA369D0EE926020E9D
:1077D000EA2207CDEEFF08CDEDFF0D010A6B00D0C8
:0A77E000072B000E0823BDD712008E
:0677EA001C0E0001DF6F20
:1077F000E06B0001000EDD6F0D0EDE6F2FEC2EF042
:107800008CEC2EF00401000E1B6F0D0E1C6F2FD997
:107810000D01010E001901E1015110E104510B6E3F
:107820000C6A060E0B1801E10C5008E105510D6EB3
:107830000E6A040E0D1801E10E5002E0000E58D041
:10784000020E061901E1075106E116C4E9FF17C44B
:10785000EAFFEF6A14D0010E061901E1075107E1B2
:10786000010E16C4E9FF17C4EAFFEF6E08D0020E3E
:1078700016C4E9FF17C4EAFFEF6E000E39D002010B
:1078800004510D01185D32E1020105510D01195D30
:107890002DE1020106510D011A5D28E10201075197
:1078A0000D011B5D23E114C4E9FF15C4EAFF08CDF7
:1078B000EEFF09CDEEFF0ACDEEFF0BCDEEFF0CCDB6
:1078C000EEFF0DCDEEFF14C4E9FF15C4EAFF060E6E
:1078D000E926000EEA220ECDEEFF0FCDEEFF10CD11
:1078E000EEFF11CDEEFF010E03D002D0000E00D04E
:1078F0001200010E0D01006F016B026B080E036F89
:10790000060E046F040E056F04011A050BE1010E4B
:107910000D01066F076B1269136914691569166901
:10792000176914D0020E0D01066F076B18C4E9FF2A
:1079300019C4EAFFEECF12FDEECF13FDEECF14FD1A
:10794000EECF15FDEECF16FDEFCF17FD08C208FDF7
:1079500009C209FD0AC20AFD0BC20BFD0CC20CFDD7
:107960000DC20DFD04C20EFD05C20FFD06C210FDC5
:1079700007C211FD18C4E9FF19C4EAFF060EE92683
:10798000000EEA22EF500E1902010E1536E118C45E
:10799000E9FF19C4EAFF060EE926000EEA22010EED
:1079A000E926000EEA22EF500D010F1902010F1512
:1079B00024E118C4E9FF19C4EAFF060EE926000E07
:1079C000EA22020EE926000EEA22EF500D011019FC
:1079D0000201101512E118C4E9FF19C4EAFF060EEE
:1079E000E926000EEA22030EE926000EEA22EF50F5
:1079F0000D0111190201111509E012C218FD13C27F
:107A000019FD14C21AFD15C21BFD10D018C4E9FFE0
:107A100019C4EAFF060EE926000EEA22EECF18FD91
:107A2000EECF19FDEECF1AFDEFCF1BFD0401000EC6
:107A30001B6F0D0E1C6F1BD81C0E0001EA6FEB6B49
:107A40000001060EE96F0001120EE76F0D0EE86FE0
:107A500040EC2FF01C0E0001DB6FDC6B0001000E10
:107A6000D96F0D0EDA6FF6EC2DF0A5EF2FF01BC4D9
:107A7000E9FF1CC4EAFFEECF0AF4EDCF0BF46EEC85
:107A800048F0F3CF0BF0F4CF0CF01BC4E9FF1CC49B
:107A9000EAFF0BC0EEFF0CC0EDFF1BC4E9FF1CC4E6
:107AA000EAFF020EE926000EEA22EECF0AF4EDCF3D
:107AB0000BF46EEC48F0F3CF0BF0F4CF0CF01BC4DA
:107AC000E9FF1CC4EAFF020E0BC0EBFF030E0CC063
:107AD000EBFF1BC4E9FF1CC4EAFF060EE926000EFB
:107AE000EA22EECF0AF4EDCF0BF46EEC48F0F3CFC0
:107AF0000BF0F4CF0CF01BC4E9FF1CC4EAFF060E28
:0C7B00000BC0EBFF070E0CC0EBFF1200E7
:047B0C00140E000152
:107B1000DF6FE06B0001080EDD6F0D0EDE6F2FECE6
:107B20002EF0F00E0D010815400801E0AED00F0E4A
:107B30000815040DF3500B6E0C6A140E0B5E000E4C
:107B40000C5A0BC01CFD1C51140801E29ED01C51A4
:107B500000080BE21C510001DF6FE06B00011D0EFD
:107B6000DD6F0D0EDE6F2FEC2EF012CD00FD13CD6C
:107B700001FD0D01126B136B140E0401126F136BD8
:107B80000401080E106F0D0E116FE6EC48F0F3CFF4
:107B900004FDF4CF05FD0D01041F051F1C51000855
:107BA00013E21C510401126F136B04011D0E106FC0
:107BB0000D0E116FE6EC48F0F3CF06FDF4CF07FD94
:107BC0000D01061F071F02D0066B076B040E040190
:107BD000126F136B0401040E106F0D0E116FE6ECA3
:107BE00048F0F3CF02FDF4CF03FD0301080EFE6F52
:107BF0000D0EFF6FC4D80D010251001902E10351AF
:107C0000011904E1F00E0815400801E03ED003011F
:107C1000F151F2110CE0F1C3E9FFF2C3EAFF18CD14
:107C2000EEFF19CDEEFF1ACDEEFF1BCDEEFFF3C335
:107C3000E9FFF4C3EAFF060EE926000EEA2214CD9E
:107C4000EEFF15CDEEFF16CDEEFF17CDEEFFF5C31F
:107C5000E9FFF6C3EAFF11CDEFFF0D011C510D6ED8
:107C60000E6A0D500A5D0B6E0E500B590C6E140E01
:107C70000B5E000E0C5AF7C3E9FFF8C3EAFF0BC016
:107C8000EEFF0CC0EDFF010E04D08CEC2EF0000EC8
:107C900000D012000D01450EB16FB26B140E03013E
:107CA000FC250D01B36F000E0301FD210D01B46F22
:107CB0000001FE2B000EFF23FEC0B5FDFFC0B6FD88
:107CC0000D01B76BB86B640EB96FFBC3BAFDBB6B2C
:107CD000BC6B04C2BDFD05C2BEFD06C2BFFD07C22E
:107CE000C0FDF9C3E9FFFAC3EAFF060EE926000E5C
:107CF000EA22EECFC1FDEECFC2FDEECFC3FDEFCF46
:107D0000C4FD0301B10EFE6F0D0EFF6F38D8140EC7
:107D10000401126F136B0401B10E106F0D0E116F81
:107D2000E6EC48F0F3CFBBFDF4CFBCFD140E03012D
:107D3000FC250001EA6F000E0301FD210001EB6F3D
:107D40000001E96BF9C3E9FFFAC3EAFFE9CFE7F005
:107D5000EACFE8F040EC2FF0140E0001DB6FDC6B93
:107D60000001B10ED96F0D0EDA6FF6EC2DF00B6A33
:107D70000C6A0BC0F3FF0CC0F4FF00D01200FEC36E
:107D8000E9FFFFC3EAFF020EE926000EEA22EECF6A
:107D90000AF4EDCF0BF46EEC48F0F3CF0BF0F4CF18
:107DA0000CF0FEC3E9FFFFC3EAFF020E0BC0EBFFBE
:107DB000030E0CC0EBFFFEC3E9FFFFC3EAFF040E96
:107DC000E926000EEA22EECF0AF4EDCF0BF46EECBA
:107DD00048F0F3CF0BF0F4CF0CF0FEC3E9FFFFC384
:107DE000EAFF040E0BC0EBFF050E0CC0EBFFFEC359
:107DF000E9FFFFC3EAFF0A0EE926000EEA22EECFF2
:107E00000AF4EDCF0BF46EEC48F0F3CF0BF0F4CFA7
:107E10000CF0FEC3E9FFFFC3EAFF0A0E0BC0EBFF45
:087E20000B0E0CC0EBFF120079
:087E28003F0EC716C66AC56AC9
:107E3000C68694869488C68AD1C3C8FF1200D3C36D
:107E4000D3FDD4C3D4FDC750040B01E0010E0B6E6B
:107E50001F0EC5140B1001E0F6D7C580C5B0FED7C4
:107E6000A1A602D0010E3ED0D2C3E0F338D900095A
:107E700002E0010E37D0C750040B01E0010E0B6E7B
:107E80001F0EC5140B1001E0F6D7C5BC29D0D4CD08
:107E9000E0F325D9000902E0010E24D0C750040BFD
:107EA00001E0010E0B6E1F0EC5140B1001E0F6D79A
:107EB000D3CDE0F314D9000902E0010E13D0C7506E
:107EC000040B01E0010E0B6E1F0EC5140B1001E038
:107ED000F6D7C5BC03D0000E05D004D0020E02D0E8
:107EE000020E00D01200D6C3D3F3D7C3D4F3D5C348
:107EF000D2F3A5DF0D01D56FD55102E0D55131D0B8
:107F0000A0D80D01D56FD55102E0D5512AD0C75068
:107F1000040B01E0010E0B6E1F0EC5140B1001E0E7
:107F2000F6D7C580C5B0FED7A1A602D0010E19D0E4
:107F30000301D5290301E06FD2D8000902E0010E48
:107F400010D0C750040B01E0010E0B6E1F0EC514BC
:107F50000B1001E0F6D7C5BC02D0000E02D0020E15
:107F600000D01200C750040B01E0010E0B6E1F0E73
:107F7000C5140B1001E0F6D7D8C3E0F3B0D8000960
:107F800002E0010E10D0C750040B01E0010E0B6E91
:107F90001F0EC5140B1001E0F6D7C5BC02D0000EB1
:107FA00002D0020E00D01200C750040B01E0010EF7
:107FB0000B6E1F0EC5140B1001E0F6D7C584C5B4B7
:107FC000FED7000E00D0120096D8C5B6FED7C59ACF
:107FD000C588C5B8FED7C95000D012008CD8C5B628
:107FE000FED7C58AC588C5B8FED7C584C5B4FED737
:107FF000000E00D01200DAC3D6F3DBC3D7F3D9C327
:10800000D5F371DF0D01776F775102E0775118D00A
:108010000301DE51DE0700090EE0D6DFE66E030144
:10802000DCC3E9FFDDC3EAFFDC2B000EDD23E552F4
:10803000E750EF6EEDD7D2DF0D01776F775100D0AB
:108040001200C750040B01E0010E0B6E1F0EC51489
:108050000B1001E0F6D7C584C5B4FED7A1A602D0A7
:10806000010E02D0000E00D01200C750040B01E038
:10807000010E0B6E1F0EC5140B1001E0F6D7C58064
:10808000C5B0FED7A1A603D0010E28D01DD0DFC3F6
:10809000E0F325D8000902E0010E20D0C750040B00
:1080A00001E0010E0B6E1F0EC5140B1001E0F6D798
:1080B000A1A602D0010E12D0C5BC03D00D01A96B40
:1080C00003D00D01040EA96FC584C5B4FED7A1A6C7
:1080D00002D0010E03D00D01A95100D01200E0C35F
:1080E000C9FFC6AE03D0FF0E05D004D0C7B0FED77F
:1080F000000E00D01200C586C7A0FED7C95000D020
:0281000012006B
:0E8102000301E26BE16B03010B0ED16F14EC75
:108110003FF0010E00D012000301E1A107D00B6A6D
:108120000C6A0BC0F3FF0CC0F4FF80D0200E0D01D1
:10813000746F756BE8C3E9FFE9C3EAFFEF5007E12D
:108140000B680C680BC0F3FF0CC0F4FF6FD0E8C3E2
:10815000E6FFE9C3E6FF59EC48F0E552E552F3CFFC
:10816000E8F3F4CFE9F303010F0EDE6F0301650EB0
:10817000DC6F0D0EDD6F74CDDAF375CDDBF303012B
:10818000A00ED96FFBEC3FF00D01655134E1E8C35F
:10819000E6FFE9C3E6FFF2EC47F0E552E552F3CF24
:1081A00076FD0D0176510C0802E20C0E766F7651C9
:1081B000E66EE66A680EE66E0D0EE66EE8C3E6FF52
:1081C000E9C3E6FF00EC48F0F56E060EE15EF550FF
:1081D00000090BE166CDE5F367CDE6F30301E22B81
:1081E00066CDF3FF67CDF4FF21D00F0E0D0174278C
:1081F000000E75231AD0040E655D10E1661D01E1C5
:10820000671D05E066CD74FD67CD75FD0ED00B686A
:108210000C680BC0F3FF0CC0F4FF08D00B680C68AF
:108220000BC0F3FF0CC0F4FF01D09DD71200030177
:10823000E76BE191E25101E0E2071200EAC3E3F3E8
:10824000EBC3E4F3EAC3D6F3EBC3D7F30301A00E09
:10825000D56F73EC3FF0000902E0000E01D0010E73
:1082600000D01200E4EC3FF00D01D36F0301E32BCB
:10827000000EE423030E0D01D35D09E1E4EC3FF0B1
:108280000D01D36F0301E32B000EE42306D0040E8F
:10829000D35D03E10301E369E4690D01D35100D02B
:1082A0001200EEEC3FF0E3C3F3FFE4C3F4FF00D0B1
:1082B00012000301E181200E0B6E0C6A0BC0F3FF6C
:1082C0000CC0F4FF00D01200ECC3E3F3EDC3E4F301
:1082D000ECC3E7F33F0E0301E717ECC3D3F3EDC3A1
:1082E000D4F30301A00ED26F1FEC3FF0000902E0AF
:1082F000000E01D0010E00D01200EEC3D8F3B2EC94
:108300003FF0000902E0000E14D00301E72BE32B3D
:10831000000EE423400EE75D0AE30CD8E3C3D3F379
:10832000E4C3D4F30301A00ED26F1FEC3FF0010EA3
:1083300000D012000301E76BD4EC3FF00301A00E64
:10834000DF6F35EC40F0000901E0F8D7E3C3F3FF3D
:10835000E4C3F4FF00D01200E5C3EAF3E6C3EBF395
:108360006DDF0D01C96BCA6B0D01C9CD0BF0CACD14
:108370000CF0C92B000ECA230301EF510B1802E1C8
:10838000F0510C1802E06EDFEFD78BDFE3C3F3FF91
:08839000E4C3F4FF00D0120069
:08839800080E0001DF6FE06B2D
:1083A0000001000EDD6F0D0EDE6F2FEC2EF002CD02
:1083B0002EFD03CD2FFD0D01026B036B080E040192
:1083C000126F136B0401000E106F0D0E116FE6ECAF
:1083D00048F0F3CF28FDF4CF29FD0D01281F291FF8
:1083E000080E0B6EAEC3E9FFAFC3EAFF0B50EF5EA2
:1083F000AEC3E9FFAFC3EAFFEF500001DF6FE06BF0
:10840000ACC3DDF0ADC3DEF02FEC2EF0AEC3E9FF60
:10841000AFC3EAFFEF500401126F136BACC310F44B
:10842000ADC311F4E6EC48F0F3CF2AFDF4CF2BFDF9
:108430000D012A1F2B1F040E0401126F136B040180
:10844000280E106F0D0E116FE6EC48F0F3CF2CFDE7
:10845000F4CF2DFD0301000EBE6F0D0EBF6F7DD852
:10846000AAC3E9FFABC3EAFF00CDEFFFB0C3E9FF4A
:10847000B1C3EAFF04CDEEFF05CDEDFFB2C3E9FFC6
:10848000B3C3EAFF06CDEEFF07CDEDFF0D012E5180
:108490002C1902E12F512D1902E0000E01D0010E1E
:1084A00000D012000D01016BB6C300FD026B036B1F
:1084B000BAC304FDBBC305FDBCC306FDBDC307FDB8
:1084C0000301B951E66EE66AB7C3E6FFB8C3E6FF3B
:1084D000080EE66E0D0EE66E83EC47F0F56E060EA6
:1084E000E15EF5500301000EBE6F0D0EBF6F35D873
:1084F000080E0301B9250401126F136B000E13233C
:108500000401000E106F0D0E116FE6EC48F0F3CF72
:1085100002FDF4CF03FD080E0301B9250301FC6F32
:10852000FD6B000EFD230301010EFB6FB4C3F9F3D5
:10853000B5C3FAF34AEC3EF0080E0301B925000179
:10854000DB6FDC6B000EDC230001000ED96F0D0E1B
:10855000DA6FF6EC2DF0A5EF2FF0BEC3E9FFBFC335
:10856000EAFF040EE926000EEA22EECF0AF4EDCF70
:108570000BF46EEC48F0F3CF0BF0F4CF0CF0BEC36D
:10858000E9FFBFC3EAFF040E0BC0EBFF050E0CC0F2
:10859000EBFFBEC3E9FFBFC3EAFF060EE926000EEC
:1085A000EA22EECF0AF4EDCF0BF46EEC48F0F3CFF5
:1085B0000BF0F4CF0CF0BEC3E9FFBFC3EAFF060E19
:1085C0000BC0EBFF070E0CC0EBFFBEC3E9FFBFC340
:1085D000EAFF020EE926000EEA22EECF0AF4EDCF02
:1085E0000BF46EEC48F0F3CF0BF0F4CF0CF0BEC3FD
:1085F000E9FFBFC3EAFF020E0BC0EBFF030E0CC086
:04860000EBFF12007A
:0C860400323030206F6B0D0A003232362D
:10861000205472616E7366657220436F6D706C6575
:1086200074650D0A0031323520446F6E652E0D0AD7
:1086300000313530205472616E7366657272696EF6
:108640006720646174612E2E2E0D0A0035333020B0
:108650004C6F67696E2072657175697265640D0A89
:1086600000353032204E6F7420696D706C656D6519
:108670006E7465640D0A00353030200D0A00323208
:1086800031204279650D0A00323330204C6F676724
:10869000656420696E0D0A003333312050617373B5
:1086A000776F72642072657175697265640D0A0076
:1086B0003232302052656164790D0A0041424F52D6
:1086C00000504F52540053544F52005155495400DA
:1086D00050415353005553455200485454502F3184
:1086E0002E3020353033200D0A0D0A53657276691D
:1086F000636520556E617661696C61626C650D0A17
:10870000000D0A0D0A00485454502F312E302032EB
:108710003030204F4B0D0A436F6E74656E742D74AC
:108720007970653A2000485454502F312E3020344F
:108730003034204E6F7420666F756E640D0A0D0A1A
:108740004E6F7420666F756E642E0D0A000D0A4E12
:108750006F772072756E6E696E67206170706C69DC
:10876000636174696F6E2E2E2E000D0A526561646E
:108770007920746F20646F776E6C6F6164204D5048
:10878000465320696D616765202D2055736520581B
:108790006D6F64656D2070726F746F636F6C2E0DFA
:1087A0000A000D0A44484350202620495020476CB7
:1087B00065616E696E672064697361626C65642EC1
:1087C0000D0A000D0A4448435020262049502047F6
:1087D0006C65616E696E6720656E61626C65642EA2
:1087E0000D0A000D0A44656661756C74205375624C
:1087F0006E6574204D61736B2028000D0A44656618
:1088000061756C7420476174657761792041646497
:10881000726573732028000D0A44656661756C7477
:1088200020495020416464726573732028000D0A4A
:1088300053657269616C204E756D62657220280007
:0E8840004D70537461636B20322E32302B006A
:02884E00030124
:10885000406B4181EEEC2CF03EEC4AF091EC35F0AF
:1088600088EF00F00D01010E3C6F0D013C5101E15C
:1088700004D13C6B03014051040A01E1DED0070A38
:1088800001E1A5D0050A01E190D0010A01E17BD008
:10889000050A3FE0070A34E0050A03E0010A01E0A7
:1088A000EBD000013B0EE56F0D0EE66F0001420EAE
:1088B000E36F030EE46FC3EC2EF000090EE1D3EC7E
:1088C0002DF0000909E10201046B056B066B076BD3
:1088D0000301418172EC31F0CFD00D01010E3C6FEC
:1088E0003B5104E10301020E406F09D0060E3B5DCF
:1088F00004E10301050E406F02D08CEC2EF0BCD0D9
:108900000D013C6B4BEC4AF0000902E00301406BA7
:10891000B3D003014C0EF76F030EF86F03013B0E4B
:10892000F56F0D0EF66F0301420EF36F030EF46F39
:108930000301370EF16F0D0EF26F86EC3DF000096A
:108940001DE00D01010E3C6F3B0504E10301030E28
:10895000406F13D0060E3B5D04E10301060E406F2D
:108960000CD0110E3B5D04E10301070E406F05D0F2
:108970003C6B8CEC2EF00301406B04D08CEC2EF0A1
:108980000301406B79D04CC33AF34DC33BF3030171
:10899000420E386F030E396FE0EC37F0000902E049
:1089A0000301406B0D013C6B67D04CC3B6F14DC366
:1089B000B7F10101420EB46F030EB56F8DEC06F0F6
:1089C000000902E00301406B0D013C6B55D0406B88
:1089D000290ED8804C55000E4D552CE30301700E26
:1089E000B26F030EB36F03016E0EB06F030EB16F63
:1089F00003014C0EAE6F030EAF6F03014E0EAC6F52
:108A0000030EAD6F03013B0EAA6F0D0EAB6FCCECE6
:108A100041F000090DE0080E0D013B5D06E1010E7D
:108A20003C6F0301040E406F02D00301406B02D083
:108A30000301406B8CEC2EF01FD0B3EC2DF000093D
:108A40001AE070C3BCF371C3BDF36EC3BAF36FC356
:108A5000BBF34CC3B9F303014E0EB76F030EB86FEF
:108A60000301B66B0301420EB46F030EB56F52ECF7
:108A700042F00301406B00D0F8D618EC05F083EC0F
:0E8A800031F00201FDA102D00301419112006C
:028A8E00FF0ED9
:108A9000E3CFEAFFE552FF0EE3CFE9FFE552E66AD6
:108AA000E66AD9CFE6FFDACFE6FFFC0EE124D96E05
:108AB000FF0EE220DA6EE66AE66AE66A200EEF5CF6
:108AC00006E0090EEF5C03E0EF6603D03FD0EE5006
:108AD000F5D72D0EEF5C03E1FF0EE32A03D02B0E3A
:108AE000EF5C01E1EE502F0EEF6424D03A0EEF6000
:108AF00021D0D890F90EE336FA0EE336FD0EDECF24
:108B0000E3FFFE0EDDCFE3FFD890F90EE336FA0E59
:108B1000E336D890F90EE336FA0EE336FD0EE35055
:108B2000DE26FE0EE350DD22300EEE5CDE26000E69
:108B3000DD22D9D7FF0EE3CFE8FFE85207E0F90EB8
:108B4000E31EE32AFA0ED8B4E306E31EE552E5522B
:108B5000E552FF0EE3CFDAFFE552FF0EE3CFD9FF78
:108B6000E552E1CFE9FFE2CFEAFFED52ED52EECF61
:108B7000F3FFEFCFF4FF1200D9CFE6FFDACFE6FF25
:108B8000FA0EE3CFD9FFFB0EE3CFDAFFFD0EE3527F
:108B900009E72D0EDE6EFC0EE31EE32AFD0ED8B4AF
:108BA000E306E31EE652E652E652FD0EE124E76ECE
:108BB000FF0EE220E46EE652F70EE3CFE6FFF70E7B
:108BC000E3CFE6FF2CEC46F0F90EE124E96EFF0E50
:108BD000E220EA6E1CEC46F00AE119EC46F009E1ED
:108BE0001CEC46F008E119EC46F007E108D027EC50
:108BF00046F022EC46F027EC46F022EC46F027EC5B
:108C000046F0DE6AF90EE126FF0EE222FF0EE3CF08
:108C1000DAFFE552FF0EE3CFD9FFE552FC0EE12467
:108C2000E96EFF0EE220EA6EEECFF3FFEFCFF4FF26
:108C30001200EF380F0B1200EF500F0B02E1EE5253
:108C4000D8841200EF380F0B300FDE6E1200EE509A
:108C50000F0B300FDE6E1200FC0EE3CFE9FFFD0EAE
:108C6000E3CFEAFF100EE66EEE6AEE6AEF6AD89086
:108C7000FD0EE336FE0EE336ED36ED36EF36FF0E33
:108C8000E30609E04DEC46F0EE524DEC46F0EE52B4
:108C90004DEC46F0EDD7E56E1200030EEF24E8B67A
:0C8CA000EF6E300EEF24E8BEEF6E000C0B
:048CAC004D70537440
:108CB00061636B20322E32302B00496E697469611A
:108CC0006C697A696E672E2E2E00444843502F47F8
:108CD0006C65616E696E672E2E2E00426F61726444
:108CE0002053657475702E2E2E0020202020202009
:108CF0002020202020202020202000434F4D4D41C7
:108D00004E44532E43474900494E4445582E48543B
:108D10004D00667470006D6963726F6368697000FE
:108D20000D0A0D0A0D4D434850537461636B204D7D
:108D300061737465722044656D6F204170706C6959
:108D4000636174696F6E20312E3120284D70537429
:108D500061636B20322E32302B2C20536570203211
:108D6000342032303033290D0A0D0A09313A2043BC
:108D700068616E676520426F617264207365726915
:108D8000616C206E756D6265722E0D0A09323A2093
:108D90004368616E67652064656661756C7420491F
:108DA0005020616464726573732E0D0A09333A2092
:108DB0004368616E67652064656661756C742067E1
:108DC00061746577617920616464726573732E0DD7
:108DD0000A09343A204368616E67652064656661FC
:108DE000756C74207375626E6574206D61736B2E83
:108DF0000D0A09353A20456E61626C65204448438E
:108E000050202620495020476C65616E696E672EA0
:108E10000D0A09363A2044697361626C6520444842
:108E20004350202620495020476C65616E696E676B
:108E30002E0D0A09373A20446F776E6C6F616420FB
:108E40004D50465320696D6167652E0D0A09383A09
:108E50002053617665202620517569742E0D0A0D08
:108E60000A456E7465722061206D656E75206368B9
:108E70006F6963652028312D38293A20000D0A4991
:108E80006E76616C696420696E70757420726563BA
:108E90006569766564202D20496E70757420696758
:108EA0006E6F7265642E0D0A507265737320616E69
:108EB00079206B657920746F20636F6E74696E75AD
:078EC000652E2E2E0D0A00A5
:088EC800FB0EE3CFF6FFFC0EE8
:108ED000E3CFF7FFFD0EE3CFF8FFFE0EE3CFE9FF90
:108EE000FF0EE3CFEAFFF90EE35003E1FA0EE35081
:108EF00009E0F90EE30602E2FA0EE3060900F55076
:108F0000EE5CF1E01200D9CFE6FFDACFE6FFFA0E11
:108F1000E3CFD9FFFB0EE3CFDAFFFC0EE3CFE9FF8F
:108F2000FD0EE3CFEAFFE9CFF3FFEACFF4FFF80E3F
:108F3000E35003E1F90EE35008E0F80EE30602E225
:108F4000F90EE306DECFEEFFF2D7FF0EE3CFDAFF36
:108F5000E552FF0EE3CFD9FFE5521200FB0EE3CF3F
:108F6000F6FFFC0EE3CFF7FFFD0EE3CFF8FFFE0E9A
:108F7000E3CFE9FFFF0EE3CFEAFFE9CFF3FFEACF4C
:108F8000F4FFF90EE35003E1FA0EE35009E0F90EA5
:108F9000E30602E2FA0EE3060900F5CFEEFFF1D791
:108FA0001200D9CFE6FFDACFE6FFFA0EE3CFD9FF02
:108FB000FB0EE3CFDAFFFC0EE3CFE9FFFD0EE3CFBC
:108FC000EAFFE9CFF3FFEACFF4FFDECFEFFFEE6673
:108FD000FCD7FF0EE3CFDAFFE552FF0EE3CFD9FF58
:108FE000E5521200FE0EE3CFE9FFFF0EE3CFEAFFEA
:108FF000F36AF46AEE5203E0F34AF42AFBD7120054
:10900000D9CFE6FFDACFE6FFFA0EE3CFD9FFFB0EAA
:10901000E3CFDAFFFC0EE3CFE9FFFD0EE3CFEAFF7B
:10902000F80EE35003E1F90EE3500AE0F80EE30610
:1090300002E2F90EE306DE50EF5C02E1EE66F0D7E5
:10904000F36EFF0EE3CFDAFFE552FF0EE3CFD9FF59
:10905000E552F3501200D9CFE6FFDACFE6FFFA0E61
:10906000E3CFD9FFFB0EE3CFDAFFFC0EE3CFE9FF3E
:10907000FD0EE3CFEAFFE9CFF3FFEACFF4FFF80EEE
:10908000E35003E1F90EE3500BE0F80EE30602E2D1
:10909000F90EE306DECFEFFFEE66F1D7DD52EFD734
:1090A000FF0EE3CFDAFFE552FF0EE3CFD9FFE55223
:1090B0001200FE0EE3CFE9FFFF0EE3CFEAFFE9CF98
:1090C000F3FFEACFF4FF610EEF5C05E67B0EEF5C89
:0C90D00002E7DF0EEF16EE52F6E1120090
:0490DC000AC4D3FDF2
:1090E0000BC4D4FDD4CDD5FDD3CDD4FDD5CDD3FD8A
:1090F000D3CDF3FFD4CDF4FF00D01200D9CFE6FFDB
:10910000E1CFD9FF0CC48CFD0DC48DFD0EC48EFDC6
:109110000FC48FFD0D018C0E906F0D0E916F90CDD1
:10912000E9FF91CDEAFF030EE926000EEA22EFCF18
:109130008BFD90CDE9FF91CDEAFFEF50E66E90CD2B
:10914000E9FF91CDEAFF030EE926000EEA22E5527F
:10915000E750EF6E90CDE9FF91CDEAFF8BCDEFFFA9
:1091600090CDE9FF91CDEAFF020EE926000EEA223A
:10917000EFCF8BFD90CDE9FF91CDEAFF010EE926FF
:10918000000EEA22EF50E66E90CDE9FF91CDEAFFA6
:10919000020EE926000EEA22E552E750EF6E90CD6E
:1091A000E9FF91CDEAFF010EE926000EEA228BCD00
:1091B000EFFF8CCD04F08DCD05F08ECD06F08FCD78
:1091C00007F000D0E552E7CFD9FF12000D01DB6BAD
:1091D000DC6BDD6BDE6B12C4D3FD13C4D4FDD89001
:1091E000D433D33310C4D5FD11C4D6FDD3CD0BF089
:1091F000D4CD0CF0D307000ED45B0B500C1018E04C
:10920000D5CDE9FFD6CDEAFF020ED527000ED62335
:10921000EECF0BF0EFCF0CF000010B510D01DB276F
:1092200000010C510D01DC23000EDD23DE23DED70F
:1092300004011251010B0EE0D5CDE9FFD6CDEAFFB6
:10924000EFCF0BF000010B510D01DB27000EDC23EB
:10925000DD23DE23DBCDD7FDDCCDD8FDDDCDD9FD93
:10926000DECDDAFDD9CDD3FDDACDD4FD0D01D95156
:10927000DA1123E0DD6BDE6BDBCD0BF0DCCD0CF027
:109280000D6A0E6AD3CD0FF0D4CD10F0116A126AB8
:109290000B500F24DB6F0C501020DC6F0D50112091
:1092A000DD6F0E501220DE6FDBCDD7FDDCCDD8FD9B
:1092B000DDCDD9FDDECDDAFDD5D7DBCD0BF0DCCDB4
:1092C0000CF00B1E0C1E0BC0F3FF0CC0F4FF00D003
:0292D00012008A
:0E92D200F00E83160F0E9512959A9598929AAB
:1092E000839A8398809AADEC27F0F00E951683163A
:1092F0008382808AB9EC27F0809AB3EC27F0F00ED5
:1093000083168382808AB9EC27F0809AB9EC27F023
:10931000F00E83168382808AB9EC27F0809A0F0EB4
:1093200095120401280E256F1AD80401280E256F06
:1093300016D80401080E256F12D804010C0E256FF3
:109340000ED80401010E256F0AD80401130E256FF3
:1093500006D80401800E256F02D800D0120024D850
:10936000000901E0FCD7959A9598F00E95168316A2
:10937000040125390F0B8312839A8398B9EC27F0E7
:10938000808AB9EC27F0809AF00E83160F0E040144
:1093900025158312B9EC27F0808AB9EC27F0809A62
:1093A0000F0E951200D01200838A8398959A959893
:1093B000B9EC27F0808AB9EC27F083A60BD0809A0D
:1093C000B9EC27F0808AB9EC27F0809A839A010ED5
:1093D0000BD00AD0809AB9EC27F0808AB9EC27F03C
:1093E000809A839A000E00D0120026C4E9FF27C499
:1093F000EAFFEFCF0CFDEF5008E00CCD2AF418D8AF
:109400000401262B000E2723F0D7120028C4F6FFF4
:1094100029C4F7FF0800F5CF08FDF55008E008CD96
:109420002AF406D80401282B000E2923EFD71200B6
:10943000BBDF000901E0FCD7959A9598F00E9516D0
:10944000831604012A390F0B0F0B83128388839A2A
:10945000B9EC27F0808AB9EC27F0809AF00E8316D9
:109460000F0E04012A158312B9EC27F0808AB9EC9B
:0C94700027F0809A0F0E951200D0120019
:04947C000301C06BBD
:10948000C169C269C369C469C569C669C76BC86B6C
:10949000C96BCA6B12000301C05101E02BD004015B
:1094A000260E166F0D0E176F04011C0E146F0D0E95
:1094B000156FF5EC3BF0000901E12ED00D012651AE
:1094C00016E11CCDC1F31DCDC2F31ECDC3F31FCDDC
:1094D000C4F320CDC5F321CDC6F322CDC7F323CDF0
:1094E000C8F324CDC9F325CDCAF316D003D00301A8
:1094F000010EC06FB3EC2DF000090CE004011A6BF3
:1095000004011C0E186F0D0E196F79EC3CF003016D
:10951000C06B02D0000E02D0010E00D01200CBC3EF
:10952000E9FFCCC3EAFFEECF22FDEECF23FDEECF65
:1095300024FDEFCF25FD0401010E1A6F04011C0E5E
:10954000186F0D0E196F79EF3CF0CDC3E9FFCEC354
:10955000EAFF0301C751EE1809E1C851EE1806E110
:10956000C951EE1803E1CA51EE1800E114E00201FE
:1095700012510301C75D21E1020113510301C85DCE
:109580001CE1020114510301C95D17E102011551EB
:109590000301CA5D12E1CFC3E9FFD0C3EAFFC1C333
:1095A000EEFFC2C3EEFFC3C3EEFFC4C3EEFFC5C3ED
:1095B000EEFFC6C3EEFF010E02D0000E00D0120077
:1095C0005458540048544D00474946004347490009
:1095D0004A504700434C4100574156007465787427
:1095E0002F706C61696E0000000000000000000038
:1095F000746578742F68746D6C00000000000000C2
:1096000000000000696D6167652F676966000000F2
:109610000000000000000000746578742F68746D0D
:109620006C0000000000000000000000696D616730
:10963000652F6A70656700000000000000000000F0
:109640006170706C69636174696F6E2F6A617661B5
:109650002D766D00617564696F2F782D7761766561
:109660000000000000000000485454502F312E30FC
:1096700020323030204F4B0D0A436F6E74656E748C
:109680002D747970653A20000D0A0D0A0047455483
:0B96900000494E4445582E48544D0040
:04969C002A0EF66E2E
:1096A000000EF76E000EF86E04010900F550056F0C
:1096B0000900F550066F03E1056701D03DD00900B0
:1096C000F550006F0900F550016F0900F550026F69
:1096D00009000900F550E96E0900F550EA6E09002D
:1096E00009000900F550036F0900F550046F0900E7
:1096F0000900F6CF07F4F7CF08F4F8CF09F400C457
:10970000F6FF01C4F7FF02C4F8FF0401035302E1AE
:10971000045307E00900F550EE6E0307F8E2040772
:10972000F9D707C4F6FF08C4F7FF09C4F8FF04011E
:0A9730000507000E065BBFD712000C
:06973A003C0ED66ED7685C
:10974000070ED56ED58EF284F28A1200D9CFE6FFCD
:10975000E1CFD9FF2BC404F02CC405F02DC406F0D2
:109760002EC407F000D0E552E7CFD9FF1200F2A4D3
:109770000AD0D7683C0ED66E04012B2B000E2C238A
:089780002D232E23F2941200A8
:08978800FF0EE350136E480EC2
:1097900001D04C0EE76EE72EFED7E76AE72EFED724
:0897A000132EF7D700001200A0
:0897A8001EEE00F02EEE00F0B1
:1097B000F86A0A9CA68EA69C4EEC4BF02EEC1EF08E
:0497C000FDD71200BF
:0C97C400FF0EE350E84E1200000000D041
:0A97D00000D000D0E82EFAD71200F6
:0697DA000201020202047C
:0E97E00004FF04FF400441044304420406FF5A
:0297EE00000079
:0897F000268706870187DA864F
:0897F800D586D086CB86C6861B
:10980000C186BC86B086988688867E867786618685
:0A9810004C86318625860D860486FD
:04981A0000FF00004B
:02981E00000048
:02982000000046
:0E9822004D70537461636B20322E32302B0078
:1098300000000D0200000000000000000000000019
:109840000000000000000000000000000000000018
:1098500000000000000000002E881788FB87E387C7
:08986000C387A2876A874D87C8
:00000001FF
